Component: ARM Compiler 5.06 update 3 (build 300) Tool: armlink [4d35c9]

==============================================================================

Section Cross References

    main.o(.text) refers to lt738_lib.o(.text) for LT738_DrawSquare_Fill
    main.o(.text) refers to gt9147.o(.text) for GT9147_Scan
    main.o(.text) refers to delay.o(.text) for delay_ms
    main.o(.text) refers to misc.o(.text) for NVIC_PriorityGroupConfig
    main.o(.text) refers to usart.o(.text) for uart_init
    main.o(.text) refers to led.o(.text) for LED_Init
    main.o(.text) refers to key.o(.text) for KEY_Init
    main.o(.text) refers to if_port.o(.text) for Parallel_Init
    main.o(.text) refers to lt738.o(.text) for Display_ON
    main.o(.text) refers to touch.o(.data) for tp_dev
    main.o(.text) refers to main.o(.constdata) for POINT_COLOR_TBL
    main.o(.text) refers to lt738_demo.o(.text) for GRAY_32
    main.o(.text) refers to gimage_home480272.o(.constdata) for gImage_home480272
    system_stm32f4xx.o(.text) refers to system_stm32f4xx.o(.data) for SystemCoreClock
    led.o(.text) refers to stm32f4xx_rcc.o(.text) for RCC_AHB1PeriphClockCmd
    led.o(.text) refers to stm32f4xx_gpio.o(.text) for GPIO_Init
    key.o(.text) refers to stm32f4xx_rcc.o(.text) for RCC_AHB1PeriphClockCmd
    key.o(.text) refers to stm32f4xx_gpio.o(.text) for GPIO_Init
    key.o(.text) refers to delay.o(.text) for delay_ms
    key.o(.text) refers to key.o(.data) for key_up
    if_port.o(.text) refers to _printf_percent.o(.ARM.Collect$$_printf_percent$$00000000) for _printf_percent
    if_port.o(.text) refers to _printf_x.o(.ARM.Collect$$_printf_percent$$0000000C) for _printf_x
    if_port.o(.text) refers to _printf_hex_int.o(.text) for _printf_longlong_hex
    if_port.o(.text) refers to stm32f4xx_rcc.o(.text) for RCC_AHB1PeriphClockCmd
    if_port.o(.text) refers to stm32f4xx_gpio.o(.text) for GPIO_Init
    if_port.o(.text) refers to stm32f4xx_fsmc.o(.text) for FSMC_NORSRAMInit
    if_port.o(.text) refers to noretval__2printf.o(.text) for __2printf
    myiic.o(.text) refers to stm32f4xx_rcc.o(.text) for RCC_AHB1PeriphClockCmd
    myiic.o(.text) refers to stm32f4xx_gpio.o(.text) for GPIO_Init
    myiic.o(.text) refers to delay.o(.text) for delay_us
    24cxx.o(.text) refers to myiic.o(.text) for IIC_Init
    24cxx.o(.text) refers to delay.o(.text) for delay_ms
    ctiic.o(.text) refers to delay.o(.text) for delay_us
    ctiic.o(.text) refers to stm32f4xx_rcc.o(.text) for RCC_AHB1PeriphClockCmd
    ctiic.o(.text) refers to stm32f4xx_gpio.o(.text) for GPIO_Init
    gt5668.o(.text) refers to _printf_percent.o(.ARM.Collect$$_printf_percent$$00000000) for _printf_percent
    gt5668.o(.text) refers to _printf_x.o(.ARM.Collect$$_printf_percent$$0000000C) for _printf_x
    gt5668.o(.text) refers to _printf_hex_int.o(.text) for _printf_longlong_hex
    gt5668.o(.text) refers to _printf_s.o(.ARM.Collect$$_printf_percent$$00000014) for _printf_s
    gt5668.o(.text) refers to _printf_str.o(.text) for _printf_str
    gt5668.o(.text) refers to _printf_pad.o(.text) for _printf_pre_padding
    gt5668.o(.text) refers to _printf_d.o(.ARM.Collect$$_printf_percent$$00000009) for _printf_d
    gt5668.o(.text) refers to _printf_dec.o(.text) for _printf_int_dec
    gt5668.o(.text) refers to noretval__2printf.o(.text) for __2printf
    gt5668.o(.text) refers to ctiic.o(.text) for CT_IIC_Start
    gt5668.o(.text) refers to rt_memclr_w.o(.text) for __aeabi_memclr4
    gt5668.o(.text) refers to stm32f4xx_rcc.o(.text) for RCC_AHB1PeriphClockCmd
    gt5668.o(.text) refers to stm32f4xx_gpio.o(.text) for GPIO_Init
    gt5668.o(.text) refers to delay.o(.text) for delay_ms
    gt5668.o(.text) refers to strcmpv7m.o(.text) for strcmp
    gt5668.o(.text) refers to gt5668.o(.constdata) for GT5668_CFG_TBL
    gt5668.o(.text) refers to gt5668.o(.data) for t
    gt5668.o(.text) refers to touch.o(.data) for tp_dev
    touch.o(.text) refers to delay.o(.text) for delay_us
    touch.o(.text) refers to lt738_lib.o(.text) for LT738_DrawLine
    touch.o(.text) refers to touch.o(.data) for CMD_RDX
    touch.o(.text) refers to touch.o(.constdata) for asc2_1206
    touch.o(.text) refers to 24cxx.o(.text) for AT24CXX_WriteLenByte
    touch.o(.text) refers to touch.o(.conststring) for .conststring
    touch.o(.text) refers to dflt_clz.o(x$fpl$dfltu) for __aeabi_ui2d
    touch.o(.text) refers to sqrt.o(i.__hardfp_sqrt) for __hardfp_sqrt
    touch.o(.text) refers to dfixu.o(x$fpl$dfixu) for __aeabi_d2uiz
    touch.o(.text) refers to f2d.o(x$fpl$f2d) for __aeabi_f2d
    touch.o(.text) refers to dleqf.o(x$fpl$dleqf) for __aeabi_cdcmple
    touch.o(.text) refers to drleqf.o(x$fpl$drleqf) for __aeabi_cdrcmple
    touch.o(.text) refers to dmul.o(x$fpl$dmul) for __aeabi_dmul
    touch.o(.text) refers to stm32f4xx_rcc.o(.text) for RCC_AHB1PeriphClockCmd
    touch.o(.text) refers to stm32f4xx_gpio.o(.text) for GPIO_Init
    touch.o(.data) refers to touch.o(.text) for TP_Init
    ft5206.o(.text) refers to _printf_percent.o(.ARM.Collect$$_printf_percent$$00000000) for _printf_percent
    ft5206.o(.text) refers to _printf_x.o(.ARM.Collect$$_printf_percent$$0000000C) for _printf_x
    ft5206.o(.text) refers to _printf_hex_int.o(.text) for _printf_longlong_hex
    ft5206.o(.text) refers to ctiic.o(.text) for CT_IIC_Start
    ft5206.o(.text) refers to stm32f4xx_rcc.o(.text) for RCC_AHB1PeriphClockCmd
    ft5206.o(.text) refers to stm32f4xx_gpio.o(.text) for GPIO_Init
    ft5206.o(.text) refers to delay.o(.text) for delay_ms
    ft5206.o(.text) refers to noretval__2printf.o(.text) for __2printf
    ft5206.o(.text) refers to ft5206.o(.data) for t
    ft5206.o(.text) refers to touch.o(.data) for tp_dev
    ft5206.o(.text) refers to ft5206.o(.constdata) for FT5206_TPX_TBL
    lt738.o(.text) refers to if_port.o(.text) for LCD_CmdWrite
    lt738_demo.o(.text) refers to lt738.o(.text) for Graphic_Mode
    lt738_demo.o(.text) refers to if_port.o(.text) for LCD_CmdWrite
    lt738_demo.o(.text) refers to lt738_lib.o(.text) for LT738_DrawSquare_Fill
    lt738_demo.o(.text) refers to key.o(.text) for WaitKey
    lt738_lib.o(.text) refers to stm32f4xx_rcc.o(.text) for RCC_AHB1PeriphClockCmd
    lt738_lib.o(.text) refers to stm32f4xx_gpio.o(.text) for GPIO_Init
    lt738_lib.o(.text) refers to if_port.o(.text) for Delay_ms
    lt738_lib.o(.text) refers to lt738.o(.text) for LCD_RegisterWrite
    lt738_lib.o(.text) refers to lt738_lib.o(.data) for SCLK
    lt738_lib.o(.text) refers to dflt_clz.o(x$fpl$dflt) for __aeabi_i2d
    lt738_lib.o(.text) refers to ddiv.o(x$fpl$ddiv) for __aeabi_ddiv
    lt738_lib.o(.text) refers to basic.o(x$fpl$basic) for __aeabi_dneg
    lt738_lib.o(.text) refers to drleqf.o(x$fpl$drleqf) for __aeabi_cdrcmple
    lt738_lib.o(.text) refers to dleqf.o(x$fpl$dleqf) for __aeabi_cdcmple
    gt9147.o(.text) refers to _printf_percent.o(.ARM.Collect$$_printf_percent$$00000000) for _printf_percent
    gt9147.o(.text) refers to _printf_x.o(.ARM.Collect$$_printf_percent$$0000000C) for _printf_x
    gt9147.o(.text) refers to _printf_hex_int.o(.text) for _printf_longlong_hex
    gt9147.o(.text) refers to _printf_s.o(.ARM.Collect$$_printf_percent$$00000014) for _printf_s
    gt9147.o(.text) refers to _printf_str.o(.text) for _printf_str
    gt9147.o(.text) refers to _printf_d.o(.ARM.Collect$$_printf_percent$$00000009) for _printf_d
    gt9147.o(.text) refers to _printf_dec.o(.text) for _printf_int_dec
    gt9147.o(.text) refers to ctiic.o(.text) for CT_IIC_Start
    gt9147.o(.text) refers to noretval__2printf.o(.text) for __2printf
    gt9147.o(.text) refers to rt_memclr_w.o(.text) for __aeabi_memclr4
    gt9147.o(.text) refers to stm32f4xx_rcc.o(.text) for RCC_AHB1PeriphClockCmd
    gt9147.o(.text) refers to stm32f4xx_gpio.o(.text) for GPIO_Init
    gt9147.o(.text) refers to delay.o(.text) for delay_ms
    gt9147.o(.text) refers to strcmpv7m.o(.text) for strcmp
    gt9147.o(.text) refers to gt9147.o(.constdata) for GT9147_CFG_TBL
    gt9147.o(.text) refers to gt9147.o(.data) for t
    gt9147.o(.text) refers to touch.o(.data) for tp_dev
    delay.o(.text) refers to misc.o(.text) for SysTick_CLKSourceConfig
    delay.o(.text) refers to delay.o(.data) for fac_us
    usart.o(.rev16_text) refers (Special) to use_no_semi_2.o(.text) for __use_no_semihosting
    usart.o(.revsh_text) refers (Special) to use_no_semi_2.o(.text) for __use_no_semihosting
    usart.o(.text) refers (Special) to use_no_semi_2.o(.text) for __use_no_semihosting
    usart.o(.text) refers to stm32f4xx_rcc.o(.text) for RCC_AHB1PeriphClockCmd
    usart.o(.text) refers to stm32f4xx_gpio.o(.text) for GPIO_PinAFConfig
    usart.o(.text) refers to stm32f4xx_usart.o(.text) for USART_Init
    usart.o(.text) refers to misc.o(.text) for NVIC_Init
    usart.o(.text) refers to usart.o(.data) for USART_RX_STA
    usart.o(.text) refers to usart.o(.bss) for USART_RX_BUF
    usart.o(.bss) refers (Special) to use_no_semi_2.o(.text) for __use_no_semihosting
    usart.o(.data) refers (Special) to use_no_semi_2.o(.text) for __use_no_semihosting
    startup_stm32f40_41xxx.o(STACK) refers (Special) to heapauxi.o(.text) for __use_two_region_memory
    startup_stm32f40_41xxx.o(HEAP) refers (Special) to heapauxi.o(.text) for __use_two_region_memory
    startup_stm32f40_41xxx.o(RESET) refers (Special) to heapauxi.o(.text) for __use_two_region_memory
    startup_stm32f40_41xxx.o(RESET) refers to startup_stm32f40_41xxx.o(STACK) for __initial_sp
    startup_stm32f40_41xxx.o(RESET) refers to startup_stm32f40_41xxx.o(.text) for Reset_Handler
    startup_stm32f40_41xxx.o(RESET) refers to stm32f4xx_it.o(.text) for NMI_Handler
    startup_stm32f40_41xxx.o(RESET) refers to usart.o(.text) for USART1_IRQHandler
    startup_stm32f40_41xxx.o(.text) refers (Special) to heapauxi.o(.text) for __use_two_region_memory
    startup_stm32f40_41xxx.o(.text) refers to system_stm32f4xx.o(.text) for SystemInit
    startup_stm32f40_41xxx.o(.text) refers to __main.o(!!!main) for __main
    startup_stm32f40_41xxx.o(.text) refers to startup_stm32f40_41xxx.o(HEAP) for Heap_Mem
    startup_stm32f40_41xxx.o(.text) refers to startup_stm32f40_41xxx.o(STACK) for Stack_Mem
    stm32f4xx_gpio.o(.text) refers to stm32f4xx_rcc.o(.text) for RCC_AHB1PeriphResetCmd
    stm32f4xx_fsmc.o(.text) refers to stm32f4xx_fsmc.o(.constdata) for FSMC_DefaultTimingStruct
    stm32f4xx_rcc.o(.text) refers to stm32f4xx_rcc.o(.data) for APBAHBPrescTable
    stm32f4xx_syscfg.o(.text) refers to stm32f4xx_rcc.o(.text) for RCC_APB2PeriphResetCmd
    stm32f4xx_usart.o(.text) refers to stm32f4xx_rcc.o(.text) for RCC_APB2PeriphResetCmd
    use_no_semi_2.o(.text) refers (Special) to use_no_semi.o(.text) for __use_no_semihosting_swi
    __2printf.o(.text) refers to _printf_char_file.o(.text) for _printf_char_file
    __2printf.o(.text) refers to usart.o(.data) for __stdout
    noretval__2printf.o(.text) refers to _printf_char_file.o(.text) for _printf_char_file
    noretval__2printf.o(.text) refers to usart.o(.data) for __stdout
    __printf.o(.text) refers to _printf_percent.o(.ARM.Collect$$_printf_percent$$00000000) for _printf_percent
    _printf_str.o(.text) refers (Special) to _printf_char.o(.text) for _printf_cs_common
    _printf_str.o(.text) refers (Weak) to _printf_pad.o(.text) for _printf_pre_padding
    _printf_str.o(.text) refers (Weak) to _printf_pad.o(.text) for _printf_post_padding
    _printf_dec.o(.text) refers to _printf_intcommon.o(.text) for _printf_int_common
    _printf_hex_ll.o(.text) refers to _printf_intcommon.o(.text) for _printf_int_common
    _printf_hex_ll.o(.text) refers to _printf_hex_ll.o(.constdata) for .constdata
    _printf_hex_int.o(.text) refers to _printf_intcommon.o(.text) for _printf_int_common
    _printf_hex_int.o(.text) refers to _printf_hex_int.o(.constdata) for .constdata
    _printf_hex_int_ll.o(.text) refers to _printf_intcommon.o(.text) for _printf_int_common
    _printf_hex_int_ll.o(.text) refers to _printf_hex_int_ll.o(.constdata) for .constdata
    _printf_hex_ptr.o(.text) refers to _printf_intcommon.o(.text) for _printf_int_common
    _printf_hex_ptr.o(.text) refers to _printf_hex_ptr.o(.constdata) for .constdata
    _printf_hex_int_ptr.o(.text) refers to _printf_intcommon.o(.text) for _printf_int_common
    _printf_hex_int_ptr.o(.text) refers to _printf_hex_int_ptr.o(.constdata) for .constdata
    _printf_hex_ll_ptr.o(.text) refers to _printf_intcommon.o(.text) for _printf_int_common
    _printf_hex_ll_ptr.o(.text) refers to _printf_hex_ll_ptr.o(.constdata) for .constdata
    _printf_hex_int_ll_ptr.o(.text) refers to _printf_intcommon.o(.text) for _printf_int_common
    _printf_hex_int_ll_ptr.o(.text) refers to _printf_hex_int_ll_ptr.o(.constdata) for .constdata
    __printf_flags.o(.text) refers to _printf_percent.o(.ARM.Collect$$_printf_percent$$00000000) for _printf_percent
    __printf_flags.o(.text) refers to __printf_flags.o(.constdata) for .constdata
    __printf_ss.o(.text) refers to _printf_percent.o(.ARM.Collect$$_printf_percent$$00000000) for _printf_percent
    __printf_flags_ss.o(.text) refers to _printf_percent.o(.ARM.Collect$$_printf_percent$$00000000) for _printf_percent
    __printf_flags_ss.o(.text) refers to __printf_flags_ss.o(.constdata) for .constdata
    __printf_wp.o(.text) refers to __printf_wp.o(i._is_digit) for _is_digit
    __printf_wp.o(.text) refers to _printf_percent.o(.ARM.Collect$$_printf_percent$$00000000) for _printf_percent
    __printf_flags_wp.o(.text) refers to __printf_wp.o(i._is_digit) for _is_digit
    __printf_flags_wp.o(.text) refers to _printf_percent.o(.ARM.Collect$$_printf_percent$$00000000) for _printf_percent
    __printf_flags_wp.o(.text) refers to __printf_flags_wp.o(.constdata) for .constdata
    __printf_ss_wp.o(.text) refers to __printf_wp.o(i._is_digit) for _is_digit
    __printf_ss_wp.o(.text) refers to _printf_percent.o(.ARM.Collect$$_printf_percent$$00000000) for _printf_percent
    __printf_flags_ss_wp.o(.text) refers to __printf_wp.o(i._is_digit) for _is_digit
    __printf_flags_ss_wp.o(.text) refers to _printf_percent.o(.ARM.Collect$$_printf_percent$$00000000) for _printf_percent
    __printf_flags_ss_wp.o(.text) refers to __printf_flags_ss_wp.o(.constdata) for .constdata
    _printf_s.o(.ARM.Collect$$_printf_percent$$00000014) refers (Weak) to _printf_char.o(.text) for _printf_string
    _printf_x.o(.ARM.Collect$$_printf_percent$$0000000C) refers (Weak) to _printf_hex_int.o(.text) for _printf_int_hex
    _printf_d.o(.ARM.Collect$$_printf_percent$$00000009) refers (Weak) to _printf_dec.o(.text) for _printf_int_dec
    _printf_percent.o(.ARM.Collect$$_printf_percent$$00000000) refers (Special) to _printf_percent_end.o(.ARM.Collect$$_printf_percent$$00000017) for _printf_percent_end
    __main.o(!!!main) refers to __rtentry.o(.ARM.Collect$$rtentry$$00000000) for __rt_entry
    basic.o(x$fpl$basic) refers (Special) to usenofp.o(x$fpl$usenofp) for __I$use$fp
    ddiv.o(x$fpl$drdiv) refers (Special) to usenofp.o(x$fpl$usenofp) for __I$use$fp
    ddiv.o(x$fpl$drdiv) refers to ddiv.o(x$fpl$ddiv) for ddiv_entry
    ddiv.o(x$fpl$ddiv) refers (Special) to usenofp.o(x$fpl$usenofp) for __I$use$fp
    ddiv.o(x$fpl$ddiv) refers to dretinf.o(x$fpl$dretinf) for __fpl_dretinf
    ddiv.o(x$fpl$ddiv) refers to dnaninf.o(x$fpl$dnaninf) for __fpl_dnaninf
    dfixu.o(x$fpl$dfixu) refers (Special) to usenofp.o(x$fpl$usenofp) for __I$use$fp
    dfixu.o(x$fpl$dfixu) refers to dnaninf.o(x$fpl$dnaninf) for __fpl_dnaninf
    dfixu.o(x$fpl$dfixur) refers (Special) to usenofp.o(x$fpl$usenofp) for __I$use$fp
    dfixu.o(x$fpl$dfixur) refers to dnaninf.o(x$fpl$dnaninf) for __fpl_dnaninf
    dflt_clz.o(x$fpl$dfltu) refers (Special) to usenofp.o(x$fpl$usenofp) for __I$use$fp
    dflt_clz.o(x$fpl$dflt) refers (Special) to usenofp.o(x$fpl$usenofp) for __I$use$fp
    dflt_clz.o(x$fpl$dfltn) refers (Special) to usenofp.o(x$fpl$usenofp) for __I$use$fp
    dleqf.o(x$fpl$dleqf) refers (Special) to usenofp.o(x$fpl$usenofp) for __I$use$fp
    dleqf.o(x$fpl$dleqf) refers to dnaninf.o(x$fpl$dnaninf) for __fpl_dnaninf
    dleqf.o(x$fpl$dleqf) refers to dcmpi.o(x$fpl$dcmpinf) for __fpl_dcmp_Inf
    dmul.o(x$fpl$dmul) refers (Special) to usenofp.o(x$fpl$usenofp) for __I$use$fp
    dmul.o(x$fpl$dmul) refers to dretinf.o(x$fpl$dretinf) for __fpl_dretinf
    dmul.o(x$fpl$dmul) refers to dnaninf.o(x$fpl$dnaninf) for __fpl_dnaninf
    drleqf.o(x$fpl$drleqf) refers (Special) to usenofp.o(x$fpl$usenofp) for __I$use$fp
    drleqf.o(x$fpl$drleqf) refers to dleqf.o(x$fpl$dleqf) for __fpl_dcmple_InfNaN
    f2d.o(x$fpl$f2d) refers (Special) to usenofp.o(x$fpl$usenofp) for __I$use$fp
    f2d.o(x$fpl$f2d) refers to fnaninf.o(x$fpl$fnaninf) for __fpl_fnaninf
    f2d.o(x$fpl$f2d) refers to dretinf.o(x$fpl$dretinf) for __fpl_dretinf
    sqrt.o(i.__hardfp_sqrt) refers (Special) to usenofp.o(x$fpl$usenofp) for __I$use$fp
    sqrt.o(i.__hardfp_sqrt) refers to dsqrt_umaal.o(x$fpl$dsqrt) for _dsqrt
    sqrt.o(i.__hardfp_sqrt) refers to _rserrno.o(.text) for __set_errno
    sqrt.o(i.__softfp_sqrt) refers (Special) to usenofp.o(x$fpl$usenofp) for __I$use$fp
    sqrt.o(i.__softfp_sqrt) refers to dsqrt_umaal.o(x$fpl$dsqrt) for _dsqrt
    sqrt.o(i.__softfp_sqrt) refers to _rserrno.o(.text) for __set_errno
    sqrt.o(i.sqrt) refers (Special) to usenofp.o(x$fpl$usenofp) for __I$use$fp
    sqrt.o(i.sqrt) refers to dsqrt_umaal.o(x$fpl$dsqrt) for _dsqrt
    sqrt.o(i.sqrt) refers to _rserrno.o(.text) for __set_errno
    sqrt_x.o(i.____hardfp_sqrt$lsc) refers (Special) to usenofp.o(x$fpl$usenofp) for __I$use$fp
    sqrt_x.o(i.____hardfp_sqrt$lsc) refers to dleqf.o(x$fpl$dleqf) for __aeabi_cdcmple
    sqrt_x.o(i.____hardfp_sqrt$lsc) refers to _rserrno.o(.text) for __set_errno
    sqrt_x.o(i.____hardfp_sqrt$lsc) refers to dsqrt_umaal.o(x$fpl$dsqrt) for _dsqrt
    sqrt_x.o(i.____softfp_sqrt$lsc) refers (Special) to usenofp.o(x$fpl$usenofp) for __I$use$fp
    sqrt_x.o(i.____softfp_sqrt$lsc) refers to dleqf.o(x$fpl$dleqf) for __aeabi_cdcmple
    sqrt_x.o(i.____softfp_sqrt$lsc) refers to _rserrno.o(.text) for __set_errno
    sqrt_x.o(i.____softfp_sqrt$lsc) refers to dsqrt_umaal.o(x$fpl$dsqrt) for _dsqrt
    sqrt_x.o(i.__sqrt$lsc) refers (Special) to usenofp.o(x$fpl$usenofp) for __I$use$fp
    sqrt_x.o(i.__sqrt$lsc) refers to dleqf.o(x$fpl$dleqf) for __aeabi_cdcmple
    sqrt_x.o(i.__sqrt$lsc) refers to _rserrno.o(.text) for __set_errno
    sqrt_x.o(i.__sqrt$lsc) refers to dsqrt_umaal.o(x$fpl$dsqrt) for _dsqrt
    __rtentry.o(.ARM.Collect$$rtentry$$00000000) refers (Special) to __rtentry2.o(.ARM.Collect$$rtentry$$0000000A) for __rt_entry_li
    __rtentry.o(.ARM.Collect$$rtentry$$00000000) refers (Special) to __rtentry2.o(.ARM.Collect$$rtentry$$0000000D) for __rt_entry_main
    __rtentry.o(.ARM.Collect$$rtentry$$00000000) refers (Special) to __rtentry2.o(.ARM.Collect$$rtentry$$0000000C) for __rt_entry_postli_1
    __rtentry.o(.ARM.Collect$$rtentry$$00000000) refers (Special) to __rtentry2.o(.ARM.Collect$$rtentry$$00000009) for __rt_entry_postsh_1
    __rtentry.o(.ARM.Collect$$rtentry$$00000000) refers (Special) to __rtentry2.o(.ARM.Collect$$rtentry$$00000002) for __rt_entry_presh_1
    __rtentry.o(.ARM.Collect$$rtentry$$00000000) refers (Special) to __rtentry4.o(.ARM.Collect$$rtentry$$00000004) for __rt_entry_sh
    _rserrno.o(.text) refers to rt_errno_addr_intlibspace.o(.text) for __aeabi_errno_addr
    _printf_intcommon.o(.text) refers (Weak) to _printf_pad.o(.text) for _printf_pre_padding
    _printf_intcommon.o(.text) refers (Weak) to _printf_pad.o(.text) for _printf_pre_padding
    _printf_intcommon.o(.text) refers (Weak) to _printf_pad.o(.text) for _printf_post_padding
    _printf_char.o(.text) refers (Weak) to _printf_str.o(.text) for _printf_str
    _printf_char_file.o(.text) refers to _printf_char_common.o(.text) for _printf_char_common
    _printf_char_file.o(.text) refers to ferror.o(.text) for ferror
    _printf_char_file.o(.text) refers to usart.o(.text) for fputc
    dcmpi.o(x$fpl$dcmpinf) refers (Special) to usenofp.o(x$fpl$usenofp) for __I$use$fp
    dnaninf.o(x$fpl$dnaninf) refers (Special) to usenofp.o(x$fpl$usenofp) for __I$use$fp
    dretinf.o(x$fpl$dretinf) refers (Special) to usenofp.o(x$fpl$usenofp) for __I$use$fp
    dsqrt_umaal.o(x$fpl$dsqrt) refers (Special) to usenofp.o(x$fpl$usenofp) for __I$use$fp
    dsqrt_umaal.o(x$fpl$dsqrt) refers to dnaninf.o(x$fpl$dnaninf) for __fpl_dnaninf
    fnaninf.o(x$fpl$fnaninf) refers (Special) to usenofp.o(x$fpl$usenofp) for __I$use$fp
    __rtentry2.o(.ARM.Collect$$rtentry$$00000008) refers to boardinit2.o(.text) for _platform_post_stackheap_init
    __rtentry2.o(.ARM.Collect$$rtentry$$0000000A) refers to libinit.o(.ARM.Collect$$libinit$$00000000) for __rt_lib_init
    __rtentry2.o(.ARM.Collect$$rtentry$$0000000B) refers to boardinit3.o(.text) for _platform_post_lib_init
    __rtentry2.o(.ARM.Collect$$rtentry$$0000000D) refers to main.o(.text) for main
    __rtentry2.o(.ARM.Collect$$rtentry$$0000000D) refers to exit.o(.text) for exit
    __rtentry2.o(.ARM.exidx) refers to __rtentry2.o(.ARM.Collect$$rtentry$$00000001) for .ARM.Collect$$rtentry$$00000001
    __rtentry2.o(.ARM.exidx) refers to __rtentry2.o(.ARM.Collect$$rtentry$$00000008) for .ARM.Collect$$rtentry$$00000008
    __rtentry2.o(.ARM.exidx) refers to __rtentry2.o(.ARM.Collect$$rtentry$$0000000A) for .ARM.Collect$$rtentry$$0000000A
    __rtentry2.o(.ARM.exidx) refers to __rtentry2.o(.ARM.Collect$$rtentry$$0000000B) for .ARM.Collect$$rtentry$$0000000B
    __rtentry2.o(.ARM.exidx) refers to __rtentry2.o(.ARM.Collect$$rtentry$$0000000D) for .ARM.Collect$$rtentry$$0000000D
    __rtentry4.o(.ARM.Collect$$rtentry$$00000004) refers to sys_stackheap_outer.o(.text) for __user_setup_stackheap
    __rtentry4.o(.ARM.exidx) refers to __rtentry4.o(.ARM.Collect$$rtentry$$00000004) for .ARM.Collect$$rtentry$$00000004
    rt_errno_addr.o(.text) refers to rt_errno_addr.o(.bss) for __aeabi_errno_addr_data
    rt_errno_addr_intlibspace.o(.text) refers to libspace.o(.bss) for __libspace_start
    _printf_char_common.o(.text) refers to __printf_flags_wp.o(.text) for __printf
    libspace.o(.text) refers to libspace.o(.bss) for __libspace_start
    sys_stackheap_outer.o(.text) refers to libspace.o(.text) for __user_perproc_libspace
    sys_stackheap_outer.o(.text) refers to startup_stm32f40_41xxx.o(.text) for __user_initial_stackheap
    exit.o(.text) refers to rtexit.o(.ARM.Collect$$rtexit$$00000000) for __rt_exit
    libinit.o(.ARM.Collect$$libinit$$00000000) refers (Special) to libinit2.o(.ARM.Collect$$libinit$$0000002E) for __rt_lib_init_alloca_1
    libinit.o(.ARM.Collect$$libinit$$00000000) refers (Special) to libinit2.o(.ARM.Collect$$libinit$$0000002C) for __rt_lib_init_argv_1
    libinit.o(.ARM.Collect$$libinit$$00000000) refers (Special) to libinit2.o(.ARM.Collect$$libinit$$0000001B) for __rt_lib_init_atexit_1
    libinit.o(.ARM.Collect$$libinit$$00000000) refers (Special) to libinit2.o(.ARM.Collect$$libinit$$00000021) for __rt_lib_init_clock_1
    libinit.o(.ARM.Collect$$libinit$$00000000) refers (Special) to libinit2.o(.ARM.Collect$$libinit$$00000032) for __rt_lib_init_cpp_1
    libinit.o(.ARM.Collect$$libinit$$00000000) refers (Special) to libinit2.o(.ARM.Collect$$libinit$$00000030) for __rt_lib_init_exceptions_1
    libinit.o(.ARM.Collect$$libinit$$00000000) refers (Special) to libinit2.o(.ARM.Collect$$libinit$$00000001) for __rt_lib_init_fp_1
    libinit.o(.ARM.Collect$$libinit$$00000000) refers (Special) to libinit2.o(.ARM.Collect$$libinit$$0000001F) for __rt_lib_init_fp_trap_1
    libinit.o(.ARM.Collect$$libinit$$00000000) refers (Special) to libinit2.o(.ARM.Collect$$libinit$$00000023) for __rt_lib_init_getenv_1
    libinit.o(.ARM.Collect$$libinit$$00000000) refers (Special) to libinit2.o(.ARM.Collect$$libinit$$0000000A) for __rt_lib_init_heap_1
    libinit.o(.ARM.Collect$$libinit$$00000000) refers (Special) to libinit2.o(.ARM.Collect$$libinit$$00000011) for __rt_lib_init_lc_collate_1
    libinit.o(.ARM.Collect$$libinit$$00000000) refers (Special) to libinit2.o(.ARM.Collect$$libinit$$00000013) for __rt_lib_init_lc_ctype_1
    libinit.o(.ARM.Collect$$libinit$$00000000) refers (Special) to libinit2.o(.ARM.Collect$$libinit$$00000015) for __rt_lib_init_lc_monetary_1
    libinit.o(.ARM.Collect$$libinit$$00000000) refers (Special) to libinit2.o(.ARM.Collect$$libinit$$00000017) for __rt_lib_init_lc_numeric_1
    libinit.o(.ARM.Collect$$libinit$$00000000) refers (Special) to libinit2.o(.ARM.Collect$$libinit$$00000019) for __rt_lib_init_lc_time_1
    libinit.o(.ARM.Collect$$libinit$$00000000) refers (Special) to libinit2.o(.ARM.Collect$$libinit$$00000004) for __rt_lib_init_preinit_1
    libinit.o(.ARM.Collect$$libinit$$00000000) refers (Special) to libinit2.o(.ARM.Collect$$libinit$$0000000E) for __rt_lib_init_rand_1
    libinit.o(.ARM.Collect$$libinit$$00000000) refers (Special) to libinit2.o(.ARM.Collect$$libinit$$00000033) for __rt_lib_init_return
    libinit.o(.ARM.Collect$$libinit$$00000000) refers (Special) to libinit2.o(.ARM.Collect$$libinit$$0000001D) for __rt_lib_init_signal_1
    libinit.o(.ARM.Collect$$libinit$$00000000) refers (Special) to libinit2.o(.ARM.Collect$$libinit$$00000025) for __rt_lib_init_stdio_1
    libinit.o(.ARM.Collect$$libinit$$00000000) refers (Special) to libinit2.o(.ARM.Collect$$libinit$$0000000C) for __rt_lib_init_user_alloc_1
    rtexit.o(.ARM.Collect$$rtexit$$00000000) refers (Special) to rtexit2.o(.ARM.Collect$$rtexit$$00000004) for __rt_exit_exit
    rtexit.o(.ARM.Collect$$rtexit$$00000000) refers (Special) to rtexit2.o(.ARM.Collect$$rtexit$$00000003) for __rt_exit_ls
    rtexit.o(.ARM.Collect$$rtexit$$00000000) refers (Special) to rtexit2.o(.ARM.Collect$$rtexit$$00000002) for __rt_exit_prels_1
    rtexit.o(.ARM.exidx) refers (Special) to rtexit2.o(.ARM.Collect$$rtexit$$00000004) for __rt_exit_exit
    rtexit.o(.ARM.exidx) refers (Special) to rtexit2.o(.ARM.Collect$$rtexit$$00000003) for __rt_exit_ls
    rtexit.o(.ARM.exidx) refers (Special) to rtexit2.o(.ARM.Collect$$rtexit$$00000002) for __rt_exit_prels_1
    rtexit.o(.ARM.exidx) refers to rtexit.o(.ARM.Collect$$rtexit$$00000000) for .ARM.Collect$$rtexit$$00000000
    libinit2.o(.ARM.Collect$$libinit$$00000001) refers to fpinit.o(x$fpl$fpinit) for _fp_init
    libinit2.o(.ARM.Collect$$libinit$$00000010) refers to libinit2.o(.ARM.Collect$$libinit$$0000000F) for .ARM.Collect$$libinit$$0000000F
    libinit2.o(.ARM.Collect$$libinit$$00000012) refers to libinit2.o(.ARM.Collect$$libinit$$0000000F) for .ARM.Collect$$libinit$$0000000F
    libinit2.o(.ARM.Collect$$libinit$$00000014) refers to libinit2.o(.ARM.Collect$$libinit$$0000000F) for .ARM.Collect$$libinit$$0000000F
    libinit2.o(.ARM.Collect$$libinit$$00000016) refers to libinit2.o(.ARM.Collect$$libinit$$0000000F) for .ARM.Collect$$libinit$$0000000F
    libinit2.o(.ARM.Collect$$libinit$$00000018) refers to libinit2.o(.ARM.Collect$$libinit$$0000000F) for .ARM.Collect$$libinit$$0000000F
    libinit2.o(.ARM.Collect$$libinit$$00000026) refers to argv_veneer.o(.emb_text) for __ARM_argv_veneer
    libinit2.o(.ARM.Collect$$libinit$$00000027) refers to argv_veneer.o(.emb_text) for __ARM_argv_veneer
    rtexit2.o(.ARM.Collect$$rtexit$$00000003) refers to libshutdown.o(.ARM.Collect$$libshutdown$$00000000) for __rt_lib_shutdown
    rtexit2.o(.ARM.Collect$$rtexit$$00000004) refers to usart.o(.text) for _sys_exit
    rtexit2.o(.ARM.exidx) refers to rtexit2.o(.ARM.Collect$$rtexit$$00000001) for .ARM.Collect$$rtexit$$00000001
    rtexit2.o(.ARM.exidx) refers to rtexit2.o(.ARM.Collect$$rtexit$$00000003) for .ARM.Collect$$rtexit$$00000003
    rtexit2.o(.ARM.exidx) refers to rtexit2.o(.ARM.Collect$$rtexit$$00000004) for .ARM.Collect$$rtexit$$00000004
    argv_veneer.o(.emb_text) refers to no_argv.o(.text) for __ARM_get_argv
    _get_argv_nomalloc.o(.text) refers (Special) to hrguard.o(.text) for __heap_region$guard
    _get_argv_nomalloc.o(.text) refers to defsig_rtmem_outer.o(.text) for __rt_SIGRTMEM
    _get_argv_nomalloc.o(.text) refers to sys_command.o(.text) for _sys_command_string
    libshutdown.o(.ARM.Collect$$libshutdown$$00000000) refers (Special) to libshutdown2.o(.ARM.Collect$$libshutdown$$00000002) for __rt_lib_shutdown_cpp_1
    libshutdown.o(.ARM.Collect$$libshutdown$$00000000) refers (Special) to libshutdown2.o(.ARM.Collect$$libshutdown$$00000007) for __rt_lib_shutdown_fp_trap_1
    libshutdown.o(.ARM.Collect$$libshutdown$$00000000) refers (Special) to libshutdown2.o(.ARM.Collect$$libshutdown$$0000000F) for __rt_lib_shutdown_heap_1
    libshutdown.o(.ARM.Collect$$libshutdown$$00000000) refers (Special) to libshutdown2.o(.ARM.Collect$$libshutdown$$00000010) for __rt_lib_shutdown_return
    libshutdown.o(.ARM.Collect$$libshutdown$$00000000) refers (Special) to libshutdown2.o(.ARM.Collect$$libshutdown$$0000000A) for __rt_lib_shutdown_signal_1
    libshutdown.o(.ARM.Collect$$libshutdown$$00000000) refers (Special) to libshutdown2.o(.ARM.Collect$$libshutdown$$00000004) for __rt_lib_shutdown_stdio_1
    libshutdown.o(.ARM.Collect$$libshutdown$$00000000) refers (Special) to libshutdown2.o(.ARM.Collect$$libshutdown$$0000000C) for __rt_lib_shutdown_user_alloc_1
    sys_command.o(.text) refers (Special) to use_no_semi.o(.text) for __I$use$semihosting
    sys_command.o(.text) refers (Special) to indicate_semi.o(.text) for __semihosting_library_function
    defsig_rtmem_outer.o(.text) refers to defsig_rtmem_inner.o(.text) for __rt_SIGRTMEM_inner
    defsig_rtmem_outer.o(.text) refers to defsig_exit.o(.text) for __sig_exit
    defsig_rtmem_formal.o(.text) refers to rt_raise.o(.text) for __rt_raise
    rt_raise.o(.text) refers to __raise.o(.text) for __raise
    rt_raise.o(.text) refers to usart.o(.text) for _sys_exit
    defsig_exit.o(.text) refers to usart.o(.text) for _sys_exit
    defsig_rtmem_inner.o(.text) refers to defsig_general.o(.text) for __default_signal_display
    __raise.o(.text) refers to defsig.o(CL$$defsig) for __default_signal_handler
    defsig_general.o(.text) refers to sys_wrch.o(.text) for _ttywrch
    sys_wrch.o(.text) refers (Special) to use_no_semi.o(.text) for __I$use$semihosting
    sys_wrch.o(.text) refers (Special) to indicate_semi.o(.text) for __semihosting_library_function
    defsig.o(CL$$defsig) refers to defsig_rtmem_inner.o(.text) for __rt_SIGRTMEM_inner
    defsig_abrt_inner.o(.text) refers to defsig_general.o(.text) for __default_signal_display
    defsig_fpe_inner.o(.text) refers to defsig_general.o(.text) for __default_signal_display
    defsig_rtred_inner.o(.text) refers to defsig_general.o(.text) for __default_signal_display
    defsig_stak_inner.o(.text) refers to defsig_general.o(.text) for __default_signal_display
    defsig_pvfn_inner.o(.text) refers to defsig_general.o(.text) for __default_signal_display
    defsig_cppl_inner.o(.text) refers to defsig_general.o(.text) for __default_signal_display
    defsig_segv_inner.o(.text) refers to defsig_general.o(.text) for __default_signal_display
    defsig_other.o(.text) refers to defsig_general.o(.text) for __default_signal_display


==============================================================================

Removing Unused input sections from the image.

    Removing main.o(.rev16_text), (4 bytes).
    Removing main.o(.revsh_text), (4 bytes).
    Removing stm32f4xx_it.o(.rev16_text), (4 bytes).
    Removing stm32f4xx_it.o(.revsh_text), (4 bytes).
    Removing system_stm32f4xx.o(.rev16_text), (4 bytes).
    Removing system_stm32f4xx.o(.revsh_text), (4 bytes).
    Removing led.o(.rev16_text), (4 bytes).
    Removing led.o(.revsh_text), (4 bytes).
    Removing key.o(.rev16_text), (4 bytes).
    Removing key.o(.revsh_text), (4 bytes).
    Removing if_port.o(.rev16_text), (4 bytes).
    Removing if_port.o(.revsh_text), (4 bytes).
    Removing myiic.o(.rev16_text), (4 bytes).
    Removing myiic.o(.revsh_text), (4 bytes).
    Removing 24cxx.o(.rev16_text), (4 bytes).
    Removing 24cxx.o(.revsh_text), (4 bytes).
    Removing ctiic.o(.rev16_text), (4 bytes).
    Removing ctiic.o(.revsh_text), (4 bytes).
    Removing gt5668.o(.rev16_text), (4 bytes).
    Removing gt5668.o(.revsh_text), (4 bytes).
    Removing gt5668.o(.text), (1336 bytes).
    Removing gt5668.o(.constdata), (250 bytes).
    Removing gt5668.o(.data), (1 bytes).
    Removing touch.o(.rev16_text), (4 bytes).
    Removing touch.o(.revsh_text), (4 bytes).
    Removing ft5206.o(.rev16_text), (4 bytes).
    Removing ft5206.o(.revsh_text), (4 bytes).
    Removing ft5206.o(.text), (812 bytes).
    Removing ft5206.o(.constdata), (10 bytes).
    Removing ft5206.o(.data), (1 bytes).
    Removing lt738.o(.rev16_text), (4 bytes).
    Removing lt738.o(.revsh_text), (4 bytes).
    Removing lt738_demo.o(.rev16_text), (4 bytes).
    Removing lt738_demo.o(.revsh_text), (4 bytes).
    Removing lt738_lib.o(.rev16_text), (4 bytes).
    Removing lt738_lib.o(.revsh_text), (4 bytes).
    Removing lt738_lib.o(.bss), (1034 bytes).
    Removing gt9147.o(.rev16_text), (4 bytes).
    Removing gt9147.o(.revsh_text), (4 bytes).
    Removing delay.o(.rev16_text), (4 bytes).
    Removing delay.o(.revsh_text), (4 bytes).
    Removing sys.o(.rev16_text), (4 bytes).
    Removing sys.o(.revsh_text), (4 bytes).
    Removing sys.o(.emb_text), (16 bytes).
    Removing usart.o(.rev16_text), (4 bytes).
    Removing usart.o(.revsh_text), (4 bytes).
    Removing misc.o(.rev16_text), (4 bytes).
    Removing misc.o(.revsh_text), (4 bytes).
    Removing stm32f4xx_gpio.o(.rev16_text), (4 bytes).
    Removing stm32f4xx_gpio.o(.revsh_text), (4 bytes).
    Removing stm32f4xx_fsmc.o(.rev16_text), (4 bytes).
    Removing stm32f4xx_fsmc.o(.revsh_text), (4 bytes).
    Removing stm32f4xx_rcc.o(.rev16_text), (4 bytes).
    Removing stm32f4xx_rcc.o(.revsh_text), (4 bytes).
    Removing stm32f4xx_syscfg.o(.rev16_text), (4 bytes).
    Removing stm32f4xx_syscfg.o(.revsh_text), (4 bytes).
    Removing stm32f4xx_syscfg.o(.text), (148 bytes).
    Removing stm32f4xx_usart.o(.rev16_text), (4 bytes).
    Removing stm32f4xx_usart.o(.revsh_text), (4 bytes).

59 unused section(s) (total 3808 bytes) removed from the image.

==============================================================================

Image Symbol Table

    Local Symbols

    Symbol Name                              Value     Ov Type        Size  Object(Section)

    ../clib/angel/boardlib.s                 0x00000000   Number         0  boardinit3.o ABSOLUTE
    ../clib/angel/boardlib.s                 0x00000000   Number         0  boardshut.o ABSOLUTE
    ../clib/angel/boardlib.s                 0x00000000   Number         0  boardinit1.o ABSOLUTE
    ../clib/angel/boardlib.s                 0x00000000   Number         0  boardinit2.o ABSOLUTE
    ../clib/angel/handlers.s                 0x00000000   Number         0  __scatter_copy.o ABSOLUTE
    ../clib/angel/handlers.s                 0x00000000   Number         0  __scatter_zi.o ABSOLUTE
    ../clib/angel/kernel.s                   0x00000000   Number         0  __rtentry.o ABSOLUTE
    ../clib/angel/kernel.s                   0x00000000   Number         0  rtexit.o ABSOLUTE
    ../clib/angel/kernel.s                   0x00000000   Number         0  rtexit2.o ABSOLUTE
    ../clib/angel/kernel.s                   0x00000000   Number         0  __rtentry2.o ABSOLUTE
    ../clib/angel/kernel.s                   0x00000000   Number         0  __rtentry4.o ABSOLUTE
    ../clib/angel/rt.s                       0x00000000   Number         0  rt_raise.o ABSOLUTE
    ../clib/angel/rt.s                       0x00000000   Number         0  rt_errno_addr.o ABSOLUTE
    ../clib/angel/rt.s                       0x00000000   Number         0  rt_errno_addr_intlibspace.o ABSOLUTE
    ../clib/angel/scatter.s                  0x00000000   Number         0  __scatter.o ABSOLUTE
    ../clib/angel/startup.s                  0x00000000   Number         0  __main.o ABSOLUTE
    ../clib/angel/sys.s                      0x00000000   Number         0  use_no_semi.o ABSOLUTE
    ../clib/angel/sys.s                      0x00000000   Number         0  libspace.o ABSOLUTE
    ../clib/angel/sys.s                      0x00000000   Number         0  use_no_semi_2.o ABSOLUTE
    ../clib/angel/sys.s                      0x00000000   Number         0  indicate_semi.o ABSOLUTE
    ../clib/angel/sys.s                      0x00000000   Number         0  sys_stackheap_outer.o ABSOLUTE
    ../clib/angel/sysapp.c                   0x00000000   Number         0  sys_command.o ABSOLUTE
    ../clib/angel/sysapp.c                   0x00000000   Number         0  sys_wrch.o ABSOLUTE
    ../clib/armsys.c                         0x00000000   Number         0  argv_veneer.o ABSOLUTE
    ../clib/armsys.c                         0x00000000   Number         0  argv_veneer.o ABSOLUTE
    ../clib/armsys.c                         0x00000000   Number         0  _get_argv_nomalloc.o ABSOLUTE
    ../clib/armsys.c                         0x00000000   Number         0  no_argv.o ABSOLUTE
    ../clib/fenv.c                           0x00000000   Number         0  _rserrno.o ABSOLUTE
    ../clib/heapalloc.c                      0x00000000   Number         0  hrguard.o ABSOLUTE
    ../clib/heapaux.c                        0x00000000   Number         0  heapauxi.o ABSOLUTE
    ../clib/libinit.s                        0x00000000   Number         0  libshutdown2.o ABSOLUTE
    ../clib/libinit.s                        0x00000000   Number         0  libinit.o ABSOLUTE
    ../clib/libinit.s                        0x00000000   Number         0  libinit2.o ABSOLUTE
    ../clib/libinit.s                        0x00000000   Number         0  libshutdown.o ABSOLUTE
    ../clib/memcpset.s                       0x00000000   Number         0  strcmpv7m.o ABSOLUTE
    ../clib/memcpset.s                       0x00000000   Number         0  rt_memclr_w.o ABSOLUTE
    ../clib/misc.s                           0x00000000   Number         0  printf_stubs.o ABSOLUTE
    ../clib/printf.c                         0x00000000   Number         0  _printf_hex_int_ptr.o ABSOLUTE
    ../clib/printf.c                         0x00000000   Number         0  _printf_dec.o ABSOLUTE
    ../clib/printf.c                         0x00000000   Number         0  __printf_flags_ss_wp.o ABSOLUTE
    ../clib/printf.c                         0x00000000   Number         0  __2printf.o ABSOLUTE
    ../clib/printf.c                         0x00000000   Number         0  _printf_hex_ll_ptr.o ABSOLUTE
    ../clib/printf.c                         0x00000000   Number         0  __printf_ss_wp.o ABSOLUTE
    ../clib/printf.c                         0x00000000   Number         0  __printf.o ABSOLUTE
    ../clib/printf.c                         0x00000000   Number         0  _printf_pad.o ABSOLUTE
    ../clib/printf.c                         0x00000000   Number         0  _printf_str.o ABSOLUTE
    ../clib/printf.c                         0x00000000   Number         0  _printf_hex_int_ll_ptr.o ABSOLUTE
    ../clib/printf.c                         0x00000000   Number         0  __printf_flags.o ABSOLUTE
    ../clib/printf.c                         0x00000000   Number         0  __printf_flags_ss.o ABSOLUTE
    ../clib/printf.c                         0x00000000   Number         0  _printf_char.o ABSOLUTE
    ../clib/printf.c                         0x00000000   Number         0  _printf_char_file.o ABSOLUTE
    ../clib/printf.c                         0x00000000   Number         0  _printf_intcommon.o ABSOLUTE
    ../clib/printf.c                         0x00000000   Number         0  __printf_ss.o ABSOLUTE
    ../clib/printf.c                         0x00000000   Number         0  _printf_hex_ptr.o ABSOLUTE
    ../clib/printf.c                         0x00000000   Number         0  _printf_hex_int_ll.o ABSOLUTE
    ../clib/printf.c                         0x00000000   Number         0  __printf_nopercent.o ABSOLUTE
    ../clib/printf.c                         0x00000000   Number         0  __printf_wp.o ABSOLUTE
    ../clib/printf.c                         0x00000000   Number         0  noretval__2printf.o ABSOLUTE
    ../clib/printf.c                         0x00000000   Number         0  _printf_char_common.o ABSOLUTE
    ../clib/printf.c                         0x00000000   Number         0  __printf_flags_wp.o ABSOLUTE
    ../clib/printf.c                         0x00000000   Number         0  _printf_hex_int.o ABSOLUTE
    ../clib/printf.c                         0x00000000   Number         0  _printf_hex_ll.o ABSOLUTE
    ../clib/printf_percent.s                 0x00000000   Number         0  _printf_percent.o ABSOLUTE
    ../clib/printf_percent.s                 0x00000000   Number         0  _printf_percent_end.o ABSOLUTE
    ../clib/printf_percent.s                 0x00000000   Number         0  _printf_x.o ABSOLUTE
    ../clib/printf_percent.s                 0x00000000   Number         0  _printf_s.o ABSOLUTE
    ../clib/printf_percent.s                 0x00000000   Number         0  _printf_d.o ABSOLUTE
    ../clib/signal.c                         0x00000000   Number         0  defsig_segv_inner.o ABSOLUTE
    ../clib/signal.c                         0x00000000   Number         0  defsig_other.o ABSOLUTE
    ../clib/signal.c                         0x00000000   Number         0  defsig_rtred_inner.o ABSOLUTE
    ../clib/signal.c                         0x00000000   Number         0  defsig_general.o ABSOLUTE
    ../clib/signal.c                         0x00000000   Number         0  __raise.o ABSOLUTE
    ../clib/signal.c                         0x00000000   Number         0  defsig_rtmem_inner.o ABSOLUTE
    ../clib/signal.c                         0x00000000   Number         0  defsig_exit.o ABSOLUTE
    ../clib/signal.c                         0x00000000   Number         0  defsig_rtmem_formal.o ABSOLUTE
    ../clib/signal.c                         0x00000000   Number         0  defsig_rtmem_outer.o ABSOLUTE
    ../clib/signal.c                         0x00000000   Number         0  defsig_fpe_inner.o ABSOLUTE
    ../clib/signal.c                         0x00000000   Number         0  defsig_abrt_inner.o ABSOLUTE
    ../clib/signal.c                         0x00000000   Number         0  defsig_stak_inner.o ABSOLUTE
    ../clib/signal.c                         0x00000000   Number         0  defsig_pvfn_inner.o ABSOLUTE
    ../clib/signal.c                         0x00000000   Number         0  defsig_cppl_inner.o ABSOLUTE
    ../clib/signal.s                         0x00000000   Number         0  defsig.o ABSOLUTE
    ../clib/stdio.c                          0x00000000   Number         0  ferror_locked.o ABSOLUTE
    ../clib/stdio.c                          0x00000000   Number         0  ferror.o ABSOLUTE
    ../clib/stdlib.c                         0x00000000   Number         0  exit.o ABSOLUTE
    ../fplib/basic.s                         0x00000000   Number         0  basic.o ABSOLUTE
    ../fplib/dcmpi.s                         0x00000000   Number         0  dcmpi.o ABSOLUTE
    ../fplib/ddiv.s                          0x00000000   Number         0  ddiv.o ABSOLUTE
    ../fplib/dfixu.s                         0x00000000   Number         0  dfixu.o ABSOLUTE
    ../fplib/dflt.s                          0x00000000   Number         0  dflt_clz.o ABSOLUTE
    ../fplib/dleqf.s                         0x00000000   Number         0  dleqf.o ABSOLUTE
    ../fplib/dmul.s                          0x00000000   Number         0  dmul.o ABSOLUTE
    ../fplib/dnaninf.s                       0x00000000   Number         0  dnaninf.o ABSOLUTE
    ../fplib/dretinf.s                       0x00000000   Number         0  dretinf.o ABSOLUTE
    ../fplib/drleqf.s                        0x00000000   Number         0  drleqf.o ABSOLUTE
    ../fplib/dsqrt.s                         0x00000000   Number         0  dsqrt_umaal.o ABSOLUTE
    ../fplib/f2d.s                           0x00000000   Number         0  f2d.o ABSOLUTE
    ../fplib/fnaninf.s                       0x00000000   Number         0  fnaninf.o ABSOLUTE
    ../fplib/fpinit.s                        0x00000000   Number         0  fpinit.o ABSOLUTE
    ../fplib/usenofp.s                       0x00000000   Number         0  usenofp.o ABSOLUTE
    ../mathlib/sqrt.c                        0x00000000   Number         0  sqrt.o ABSOLUTE
    ../mathlib/sqrt.c                        0x00000000   Number         0  sqrt_x.o ABSOLUTE
    ..\CORE\startup_stm32f40_41xxx.s         0x00000000   Number         0  startup_stm32f40_41xxx.o ABSOLUTE
    ..\FWLIB\src\misc.c                      0x00000000   Number         0  misc.o ABSOLUTE
    ..\FWLIB\src\stm32f4xx_fsmc.c            0x00000000   Number         0  stm32f4xx_fsmc.o ABSOLUTE
    ..\FWLIB\src\stm32f4xx_gpio.c            0x00000000   Number         0  stm32f4xx_gpio.o ABSOLUTE
    ..\FWLIB\src\stm32f4xx_rcc.c             0x00000000   Number         0  stm32f4xx_rcc.o ABSOLUTE
    ..\FWLIB\src\stm32f4xx_syscfg.c          0x00000000   Number         0  stm32f4xx_syscfg.o ABSOLUTE
    ..\FWLIB\src\stm32f4xx_usart.c           0x00000000   Number         0  stm32f4xx_usart.o ABSOLUTE
    ..\HARDWARE\24CXX\24cxx.c                0x00000000   Number         0  24cxx.o ABSOLUTE
    ..\HARDWARE\IF_PORT\if_port.c            0x00000000   Number         0  if_port.o ABSOLUTE
    ..\HARDWARE\IIC\myiic.c                  0x00000000   Number         0  myiic.o ABSOLUTE
    ..\HARDWARE\KEY\key.c                    0x00000000   Number         0  key.o ABSOLUTE
    ..\HARDWARE\LCD\gImage_home480272.c      0x00000000   Number         0  gimage_home480272.o ABSOLUTE
    ..\HARDWARE\LED\led.c                    0x00000000   Number         0  led.o ABSOLUTE
    ..\HARDWARE\LT738\LT738.c                0x00000000   Number         0  lt738.o ABSOLUTE
    ..\HARDWARE\LT738_Demo\LT738_Demo.c      0x00000000   Number         0  lt738_demo.o ABSOLUTE
    ..\HARDWARE\LT738_Lib\LT738_Lib.c        0x00000000   Number         0  lt738_lib.o ABSOLUTE
    ..\HARDWARE\TOUCH\ctiic.c                0x00000000   Number         0  ctiic.o ABSOLUTE
    ..\HARDWARE\TOUCH\ft5206.c               0x00000000   Number         0  ft5206.o ABSOLUTE
    ..\HARDWARE\TOUCH\gt5668.c               0x00000000   Number         0  gt5668.o ABSOLUTE
    ..\HARDWARE\TOUCH\gt9147.c               0x00000000   Number         0  gt9147.o ABSOLUTE
    ..\HARDWARE\TOUCH\touch.c                0x00000000   Number         0  touch.o ABSOLUTE
    ..\SYSTEM\delay\delay.c                  0x00000000   Number         0  delay.o ABSOLUTE
    ..\SYSTEM\sys\sys.c                      0x00000000   Number         0  sys.o ABSOLUTE
    ..\SYSTEM\usart\usart.c                  0x00000000   Number         0  usart.o ABSOLUTE
    ..\\FWLIB\\src\\misc.c                   0x00000000   Number         0  misc.o ABSOLUTE
    ..\\FWLIB\\src\\stm32f4xx_fsmc.c         0x00000000   Number         0  stm32f4xx_fsmc.o ABSOLUTE
    ..\\FWLIB\\src\\stm32f4xx_gpio.c         0x00000000   Number         0  stm32f4xx_gpio.o ABSOLUTE
    ..\\FWLIB\\src\\stm32f4xx_rcc.c          0x00000000   Number         0  stm32f4xx_rcc.o ABSOLUTE
    ..\\FWLIB\\src\\stm32f4xx_syscfg.c       0x00000000   Number         0  stm32f4xx_syscfg.o ABSOLUTE
    ..\\FWLIB\\src\\stm32f4xx_usart.c        0x00000000   Number         0  stm32f4xx_usart.o ABSOLUTE
    ..\\HARDWARE\\24CXX\\24cxx.c             0x00000000   Number         0  24cxx.o ABSOLUTE
    ..\\HARDWARE\\IF_PORT\\if_port.c         0x00000000   Number         0  if_port.o ABSOLUTE
    ..\\HARDWARE\\IIC\\myiic.c               0x00000000   Number         0  myiic.o ABSOLUTE
    ..\\HARDWARE\\KEY\\key.c                 0x00000000   Number         0  key.o ABSOLUTE
    ..\\HARDWARE\\LED\\led.c                 0x00000000   Number         0  led.o ABSOLUTE
    ..\\HARDWARE\\LT738\\LT738.c             0x00000000   Number         0  lt738.o ABSOLUTE
    ..\\HARDWARE\\LT738_Demo\\LT738_Demo.c   0x00000000   Number         0  lt738_demo.o ABSOLUTE
    ..\\HARDWARE\\LT738_Lib\\LT738_Lib.c     0x00000000   Number         0  lt738_lib.o ABSOLUTE
    ..\\HARDWARE\\TOUCH\\ctiic.c             0x00000000   Number         0  ctiic.o ABSOLUTE
    ..\\HARDWARE\\TOUCH\\ft5206.c            0x00000000   Number         0  ft5206.o ABSOLUTE
    ..\\HARDWARE\\TOUCH\\gt5668.c            0x00000000   Number         0  gt5668.o ABSOLUTE
    ..\\HARDWARE\\TOUCH\\gt9147.c            0x00000000   Number         0  gt9147.o ABSOLUTE
    ..\\HARDWARE\\TOUCH\\touch.c             0x00000000   Number         0  touch.o ABSOLUTE
    ..\\SYSTEM\\delay\\delay.c               0x00000000   Number         0  delay.o ABSOLUTE
    ..\\SYSTEM\\sys\\sys.c                   0x00000000   Number         0  sys.o ABSOLUTE
    ..\\SYSTEM\\usart\\usart.c               0x00000000   Number         0  usart.o ABSOLUTE
    dc.s                                     0x00000000   Number         0  dc.o ABSOLUTE
    main.c                                   0x00000000   Number         0  main.o ABSOLUTE
    main.c                                   0x00000000   Number         0  main.o ABSOLUTE
    stm32f4xx_it.c                           0x00000000   Number         0  stm32f4xx_it.o ABSOLUTE
    stm32f4xx_it.c                           0x00000000   Number         0  stm32f4xx_it.o ABSOLUTE
    system_stm32f4xx.c                       0x00000000   Number         0  system_stm32f4xx.o ABSOLUTE
    system_stm32f4xx.c                       0x00000000   Number         0  system_stm32f4xx.o ABSOLUTE
    RESET                                    0x08000000   Section      392  startup_stm32f40_41xxx.o(RESET)
    !!!main                                  0x08000188   Section        8  __main.o(!!!main)
    !!!scatter                               0x08000190   Section       52  __scatter.o(!!!scatter)
    !!handler_copy                           0x080001c4   Section       26  __scatter_copy.o(!!handler_copy)
    !!handler_zi                             0x080001e0   Section       28  __scatter_zi.o(!!handler_zi)
    .ARM.Collect$$_printf_percent$$00000000  0x080001fc   Section        0  _printf_percent.o(.ARM.Collect$$_printf_percent$$00000000)
    .ARM.Collect$$_printf_percent$$00000009  0x080001fc   Section        6  _printf_d.o(.ARM.Collect$$_printf_percent$$00000009)
    .ARM.Collect$$_printf_percent$$0000000C  0x08000202   Section        6  _printf_x.o(.ARM.Collect$$_printf_percent$$0000000C)
    .ARM.Collect$$_printf_percent$$00000014  0x08000208   Section        6  _printf_s.o(.ARM.Collect$$_printf_percent$$00000014)
    .ARM.Collect$$_printf_percent$$00000017  0x0800020e   Section        4  _printf_percent_end.o(.ARM.Collect$$_printf_percent$$00000017)
    .ARM.Collect$$libinit$$00000000          0x08000212   Section        2  libinit.o(.ARM.Collect$$libinit$$00000000)
    .ARM.Collect$$libinit$$00000001          0x08000214   Section        4  libinit2.o(.ARM.Collect$$libinit$$00000001)
    .ARM.Collect$$libinit$$00000004          0x08000218   Section        0  libinit2.o(.ARM.Collect$$libinit$$00000004)
    .ARM.Collect$$libinit$$0000000A          0x08000218   Section        0  libinit2.o(.ARM.Collect$$libinit$$0000000A)
    .ARM.Collect$$libinit$$0000000C          0x08000218   Section        0  libinit2.o(.ARM.Collect$$libinit$$0000000C)
    .ARM.Collect$$libinit$$0000000E          0x08000218   Section        0  libinit2.o(.ARM.Collect$$libinit$$0000000E)
    .ARM.Collect$$libinit$$00000011          0x08000218   Section        0  libinit2.o(.ARM.Collect$$libinit$$00000011)
    .ARM.Collect$$libinit$$00000013          0x08000218   Section        0  libinit2.o(.ARM.Collect$$libinit$$00000013)
    .ARM.Collect$$libinit$$00000015          0x08000218   Section        0  libinit2.o(.ARM.Collect$$libinit$$00000015)
    .ARM.Collect$$libinit$$00000017          0x08000218   Section        0  libinit2.o(.ARM.Collect$$libinit$$00000017)
    .ARM.Collect$$libinit$$00000019          0x08000218   Section        0  libinit2.o(.ARM.Collect$$libinit$$00000019)
    .ARM.Collect$$libinit$$0000001B          0x08000218   Section        0  libinit2.o(.ARM.Collect$$libinit$$0000001B)
    .ARM.Collect$$libinit$$0000001D          0x08000218   Section        0  libinit2.o(.ARM.Collect$$libinit$$0000001D)
    .ARM.Collect$$libinit$$0000001F          0x08000218   Section        0  libinit2.o(.ARM.Collect$$libinit$$0000001F)
    .ARM.Collect$$libinit$$00000021          0x08000218   Section        0  libinit2.o(.ARM.Collect$$libinit$$00000021)
    .ARM.Collect$$libinit$$00000023          0x08000218   Section        0  libinit2.o(.ARM.Collect$$libinit$$00000023)
    .ARM.Collect$$libinit$$00000025          0x08000218   Section        0  libinit2.o(.ARM.Collect$$libinit$$00000025)
    .ARM.Collect$$libinit$$0000002C          0x08000218   Section        0  libinit2.o(.ARM.Collect$$libinit$$0000002C)
    .ARM.Collect$$libinit$$0000002E          0x08000218   Section        0  libinit2.o(.ARM.Collect$$libinit$$0000002E)
    .ARM.Collect$$libinit$$00000030          0x08000218   Section        0  libinit2.o(.ARM.Collect$$libinit$$00000030)
    .ARM.Collect$$libinit$$00000032          0x08000218   Section        0  libinit2.o(.ARM.Collect$$libinit$$00000032)
    .ARM.Collect$$libinit$$00000033          0x08000218   Section        2  libinit2.o(.ARM.Collect$$libinit$$00000033)
    .ARM.Collect$$libshutdown$$00000000      0x0800021a   Section        2  libshutdown.o(.ARM.Collect$$libshutdown$$00000000)
    .ARM.Collect$$libshutdown$$00000002      0x0800021c   Section        0  libshutdown2.o(.ARM.Collect$$libshutdown$$00000002)
    .ARM.Collect$$libshutdown$$00000004      0x0800021c   Section        0  libshutdown2.o(.ARM.Collect$$libshutdown$$00000004)
    .ARM.Collect$$libshutdown$$00000007      0x0800021c   Section        0  libshutdown2.o(.ARM.Collect$$libshutdown$$00000007)
    .ARM.Collect$$libshutdown$$0000000A      0x0800021c   Section        0  libshutdown2.o(.ARM.Collect$$libshutdown$$0000000A)
    .ARM.Collect$$libshutdown$$0000000C      0x0800021c   Section        0  libshutdown2.o(.ARM.Collect$$libshutdown$$0000000C)
    .ARM.Collect$$libshutdown$$0000000F      0x0800021c   Section        0  libshutdown2.o(.ARM.Collect$$libshutdown$$0000000F)
    .ARM.Collect$$libshutdown$$00000010      0x0800021c   Section        2  libshutdown2.o(.ARM.Collect$$libshutdown$$00000010)
    .ARM.Collect$$rtentry$$00000000          0x0800021e   Section        0  __rtentry.o(.ARM.Collect$$rtentry$$00000000)
    .ARM.Collect$$rtentry$$00000002          0x0800021e   Section        0  __rtentry2.o(.ARM.Collect$$rtentry$$00000002)
    .ARM.Collect$$rtentry$$00000004          0x0800021e   Section        6  __rtentry4.o(.ARM.Collect$$rtentry$$00000004)
    .ARM.Collect$$rtentry$$00000009          0x08000224   Section        0  __rtentry2.o(.ARM.Collect$$rtentry$$00000009)
    .ARM.Collect$$rtentry$$0000000A          0x08000224   Section        4  __rtentry2.o(.ARM.Collect$$rtentry$$0000000A)
    .ARM.Collect$$rtentry$$0000000C          0x08000228   Section        0  __rtentry2.o(.ARM.Collect$$rtentry$$0000000C)
    .ARM.Collect$$rtentry$$0000000D          0x08000228   Section        8  __rtentry2.o(.ARM.Collect$$rtentry$$0000000D)
    .ARM.Collect$$rtexit$$00000000           0x08000230   Section        2  rtexit.o(.ARM.Collect$$rtexit$$00000000)
    .ARM.Collect$$rtexit$$00000002           0x08000232   Section        0  rtexit2.o(.ARM.Collect$$rtexit$$00000002)
    .ARM.Collect$$rtexit$$00000003           0x08000232   Section        4  rtexit2.o(.ARM.Collect$$rtexit$$00000003)
    .ARM.Collect$$rtexit$$00000004           0x08000236   Section        6  rtexit2.o(.ARM.Collect$$rtexit$$00000004)
    .text                                    0x0800023c   Section        0  main.o(.text)
    .text                                    0x080006fc   Section        0  stm32f4xx_it.o(.text)
    .text                                    0x08000718   Section        0  system_stm32f4xx.o(.text)
    SetSysClock                              0x08000719   Thumb Code   220  system_stm32f4xx.o(.text)
    .text                                    0x08000928   Section        0  led.o(.text)
    .text                                    0x08000968   Section        0  key.o(.text)
    .text                                    0x08000bf4   Section        0  if_port.o(.text)
    .text                                    0x08000f2c   Section        0  myiic.o(.text)
    .text                                    0x08001188   Section        0  24cxx.o(.text)
    .text                                    0x08001304   Section        0  ctiic.o(.text)
    .text                                    0x08001558   Section        0  touch.o(.text)
    .text                                    0x08002598   Section        0  lt738.o(.text)
    .text                                    0x080052cc   Section        0  lt738_demo.o(.text)
    .text                                    0x08005570   Section        0  lt738_lib.o(.text)
    .text                                    0x080070fc   Section        0  gt9147.o(.text)
    .text                                    0x08007570   Section        0  delay.o(.text)
    .text                                    0x08007674   Section        0  usart.o(.text)
    .text                                    0x080077bc   Section       64  startup_stm32f40_41xxx.o(.text)
    $v0                                      0x080077bc   Number         0  startup_stm32f40_41xxx.o(.text)
    .text                                    0x080077fc   Section        0  misc.o(.text)
    .text                                    0x080078dc   Section        0  stm32f4xx_gpio.o(.text)
    .text                                    0x08007b70   Section        0  stm32f4xx_fsmc.o(.text)
    .text                                    0x08008138   Section        0  stm32f4xx_rcc.o(.text)
    .text                                    0x08008794   Section        0  stm32f4xx_usart.o(.text)
    .text                                    0x08008be8   Section        2  use_no_semi_2.o(.text)
    .text                                    0x08008bec   Section        0  noretval__2printf.o(.text)
    .text                                    0x08008c04   Section        0  _printf_str.o(.text)
    .text                                    0x08008c58   Section        0  _printf_dec.o(.text)
    .text                                    0x08008cd0   Section        0  _printf_hex_int.o(.text)
    .text                                    0x08008d28   Section        0  __printf_flags_wp.o(.text)
    .text                                    0x08008e60   Section       78  rt_memclr_w.o(.text)
    .text                                    0x08008eb0   Section      128  strcmpv7m.o(.text)
    .text                                    0x08008f30   Section        0  heapauxi.o(.text)
    .text                                    0x08008f36   Section        2  use_no_semi.o(.text)
    .text                                    0x08008f38   Section        0  _rserrno.o(.text)
    .text                                    0x08008f4e   Section        0  _printf_intcommon.o(.text)
    .text                                    0x08009000   Section        0  _printf_char.o(.text)
    .text                                    0x0800902c   Section        0  _printf_char_file.o(.text)
    .text                                    0x08009050   Section        8  rt_errno_addr_intlibspace.o(.text)
    .text                                    0x08009058   Section        0  _printf_char_common.o(.text)
    _printf_input_char                       0x08009059   Thumb Code    10  _printf_char_common.o(.text)
    .text                                    0x08009088   Section        0  ferror.o(.text)
    .text                                    0x08009090   Section        8  libspace.o(.text)
    .text                                    0x08009098   Section       74  sys_stackheap_outer.o(.text)
    .text                                    0x080090e2   Section        0  exit.o(.text)
    i.__hardfp_sqrt                          0x080090f4   Section        0  sqrt.o(i.__hardfp_sqrt)
    i._is_digit                              0x0800916e   Section        0  __printf_wp.o(i._is_digit)
    x$fpl$basic                              0x0800917c   Section       24  basic.o(x$fpl$basic)
    $v0                                      0x0800917c   Number         0  basic.o(x$fpl$basic)
    x$fpl$dcmpinf                            0x08009194   Section       24  dcmpi.o(x$fpl$dcmpinf)
    $v0                                      0x08009194   Number         0  dcmpi.o(x$fpl$dcmpinf)
    x$fpl$ddiv                               0x080091ac   Section      688  ddiv.o(x$fpl$ddiv)
    $v0                                      0x080091ac   Number         0  ddiv.o(x$fpl$ddiv)
    ddiv_entry                               0x080091b3   Thumb Code     0  ddiv.o(x$fpl$ddiv)
    x$fpl$dfixu                              0x0800945c   Section       90  dfixu.o(x$fpl$dfixu)
    $v0                                      0x0800945c   Number         0  dfixu.o(x$fpl$dfixu)
    x$fpl$dflt                               0x080094b6   Section       46  dflt_clz.o(x$fpl$dflt)
    $v0                                      0x080094b6   Number         0  dflt_clz.o(x$fpl$dflt)
    x$fpl$dfltu                              0x080094e4   Section       38  dflt_clz.o(x$fpl$dfltu)
    $v0                                      0x080094e4   Number         0  dflt_clz.o(x$fpl$dfltu)
    x$fpl$dleqf                              0x0800950c   Section      120  dleqf.o(x$fpl$dleqf)
    $v0                                      0x0800950c   Number         0  dleqf.o(x$fpl$dleqf)
    x$fpl$dmul                               0x08009584   Section      340  dmul.o(x$fpl$dmul)
    $v0                                      0x08009584   Number         0  dmul.o(x$fpl$dmul)
    x$fpl$dnaninf                            0x080096d8   Section      156  dnaninf.o(x$fpl$dnaninf)
    $v0                                      0x080096d8   Number         0  dnaninf.o(x$fpl$dnaninf)
    x$fpl$dretinf                            0x08009774   Section       12  dretinf.o(x$fpl$dretinf)
    $v0                                      0x08009774   Number         0  dretinf.o(x$fpl$dretinf)
    x$fpl$drleqf                             0x08009780   Section      108  drleqf.o(x$fpl$drleqf)
    $v0                                      0x08009780   Number         0  drleqf.o(x$fpl$drleqf)
    x$fpl$dsqrt                              0x080097ec   Section      408  dsqrt_umaal.o(x$fpl$dsqrt)
    $v0                                      0x080097ec   Number         0  dsqrt_umaal.o(x$fpl$dsqrt)
    x$fpl$f2d                                0x08009984   Section       86  f2d.o(x$fpl$f2d)
    $v0                                      0x08009984   Number         0  f2d.o(x$fpl$f2d)
    x$fpl$fnaninf                            0x080099da   Section      140  fnaninf.o(x$fpl$fnaninf)
    $v0                                      0x080099da   Number         0  fnaninf.o(x$fpl$fnaninf)
    x$fpl$fpinit                             0x08009a66   Section       10  fpinit.o(x$fpl$fpinit)
    $v0                                      0x08009a66   Number         0  fpinit.o(x$fpl$fpinit)
    .constdata                               0x08009a70   Section      478  main.o(.constdata)
    x$fpl$usenofp                            0x08009a70   Section        0  usenofp.o(x$fpl$usenofp)
    .constdata                               0x08009c4e   Section     6080  touch.o(.constdata)
    .constdata                               0x0800b40e   Section    261120  gimage_home480272.o(.constdata)
    .constdata                               0x0804b00e   Section      196  gt9147.o(.constdata)
    .constdata                               0x0804b0d4   Section       28  stm32f4xx_fsmc.o(.constdata)
    .constdata                               0x0804b0f0   Section       40  _printf_hex_int.o(.constdata)
    uc_hextab                                0x0804b0f0   Data          20  _printf_hex_int.o(.constdata)
    lc_hextab                                0x0804b104   Data          20  _printf_hex_int.o(.constdata)
    .constdata                               0x0804b118   Section       17  __printf_flags_wp.o(.constdata)
    maptable                                 0x0804b118   Data          17  __printf_flags_wp.o(.constdata)
    .conststring                             0x0804b12c   Section      121  touch.o(.conststring)
    .data                                    0x20000000   Section       20  system_stm32f4xx.o(.data)
    .data                                    0x20000014   Section        2  key.o(.data)
    key_up                                   0x20000014   Data           1  key.o(.data)
    key_up                                   0x20000015   Data           1  key.o(.data)
    .data                                    0x20000018   Section       54  touch.o(.data)
    .data                                    0x2000004e   Section        3  lt738_lib.o(.data)
    .data                                    0x20000051   Section        1  gt9147.o(.data)
    t                                        0x20000051   Data           1  gt9147.o(.data)
    .data                                    0x20000052   Section        4  delay.o(.data)
    fac_us                                   0x20000052   Data           1  delay.o(.data)
    fac_ms                                   0x20000054   Data           2  delay.o(.data)
    .data                                    0x20000058   Section        6  usart.o(.data)
    .data                                    0x2000005e   Section       16  stm32f4xx_rcc.o(.data)
    APBAHBPrescTable                         0x2000005e   Data          16  stm32f4xx_rcc.o(.data)
    .bss                                     0x20000070   Section      200  usart.o(.bss)
    .bss                                     0x20000138   Section       96  libspace.o(.bss)
    HEAP                                     0x20000198   Section      512  startup_stm32f40_41xxx.o(HEAP)
    Heap_Mem                                 0x20000198   Data         512  startup_stm32f40_41xxx.o(HEAP)
    STACK                                    0x20000398   Section     1024  startup_stm32f40_41xxx.o(STACK)
    Stack_Mem                                0x20000398   Data        1024  startup_stm32f40_41xxx.o(STACK)
    __initial_sp                             0x20000798   Data           0  startup_stm32f40_41xxx.o(STACK)

    Global Symbols

    Symbol Name                              Value     Ov Type        Size  Object(Section)

    BuildAttributes$$THM_ISAv4$E$P$D$K$B$S$7EM$VFPi3$EXTD16$VFPS$VFMA$PE$A:L22UL41UL21$X:L11$S22US41US21$IEEE1$IW$USESV6$~STKCKD$USESV7$~SHL$OTIME$ROPI$IEEEJ$EBA8$UX$STANDARDLIB$REQ8$PRES8$EABIv2 0x00000000   Number         0  anon$$obj.o ABSOLUTE
    __ARM_use_no_argv                        0x00000000   Number         0  main.o ABSOLUTE
    _printf_flags                            0x00000000   Number         0  printf_stubs.o ABSOLUTE
    _printf_return_value                     0x00000000   Number         0  printf_stubs.o ABSOLUTE
    _printf_sizespec                         0x00000000   Number         0  printf_stubs.o ABSOLUTE
    _printf_widthprec                        0x00000000   Number         0  printf_stubs.o ABSOLUTE
    __ARM_exceptions_init                     - Undefined Weak Reference
    __alloca_initialize                       - Undefined Weak Reference
    __arm_preinit_                            - Undefined Weak Reference
    __cpp_initialize__aeabi_                  - Undefined Weak Reference
    __cxa_finalize                            - Undefined Weak Reference
    __rt_locale                               - Undefined Weak Reference
    __sigvec_lookup                           - Undefined Weak Reference
    _atexit_init                              - Undefined Weak Reference
    _call_atexit_fns                          - Undefined Weak Reference
    _clock_init                               - Undefined Weak Reference
    _fp_trap_init                             - Undefined Weak Reference
    _fp_trap_shutdown                         - Undefined Weak Reference
    _get_lc_collate                           - Undefined Weak Reference
    _get_lc_ctype                             - Undefined Weak Reference
    _get_lc_monetary                          - Undefined Weak Reference
    _get_lc_numeric                           - Undefined Weak Reference
    _get_lc_time                              - Undefined Weak Reference
    _getenv_init                              - Undefined Weak Reference
    _handle_redirection                       - Undefined Weak Reference
    _init_alloc                               - Undefined Weak Reference
    _init_user_alloc                          - Undefined Weak Reference
    _initio                                   - Undefined Weak Reference
    _mutex_acquire                            - Undefined Weak Reference
    _mutex_release                            - Undefined Weak Reference
    _printf_mbtowc                            - Undefined Weak Reference
    _printf_truncate_signed                   - Undefined Weak Reference
    _printf_truncate_unsigned                 - Undefined Weak Reference
    _rand_init                                - Undefined Weak Reference
    _signal_finish                            - Undefined Weak Reference
    _signal_init                              - Undefined Weak Reference
    _terminate_alloc                          - Undefined Weak Reference
    _terminate_user_alloc                     - Undefined Weak Reference
    _terminateio                              - Undefined Weak Reference
    __Vectors_Size                           0x00000188   Number         0  startup_stm32f40_41xxx.o ABSOLUTE
    __Vectors                                0x08000000   Data           4  startup_stm32f40_41xxx.o(RESET)
    __Vectors_End                            0x08000188   Data           0  startup_stm32f40_41xxx.o(RESET)
    __main                                   0x08000189   Thumb Code     8  __main.o(!!!main)
    __scatterload                            0x08000191   Thumb Code     0  __scatter.o(!!!scatter)
    __scatterload_rt2                        0x08000191   Thumb Code    44  __scatter.o(!!!scatter)
    __scatterload_rt2_thumb_only             0x08000191   Thumb Code     0  __scatter.o(!!!scatter)
    __scatterload_null                       0x0800019f   Thumb Code     0  __scatter.o(!!!scatter)
    __scatterload_copy                       0x080001c5   Thumb Code    26  __scatter_copy.o(!!handler_copy)
    __scatterload_zeroinit                   0x080001e1   Thumb Code    28  __scatter_zi.o(!!handler_zi)
    _printf_d                                0x080001fd   Thumb Code     0  _printf_d.o(.ARM.Collect$$_printf_percent$$00000009)
    _printf_percent                          0x080001fd   Thumb Code     0  _printf_percent.o(.ARM.Collect$$_printf_percent$$00000000)
    _printf_x                                0x08000203   Thumb Code     0  _printf_x.o(.ARM.Collect$$_printf_percent$$0000000C)
    _printf_s                                0x08000209   Thumb Code     0  _printf_s.o(.ARM.Collect$$_printf_percent$$00000014)
    _printf_percent_end                      0x0800020f   Thumb Code     0  _printf_percent_end.o(.ARM.Collect$$_printf_percent$$00000017)
    __rt_lib_init                            0x08000213   Thumb Code     0  libinit.o(.ARM.Collect$$libinit$$00000000)
    __rt_lib_init_fp_1                       0x08000215   Thumb Code     0  libinit2.o(.ARM.Collect$$libinit$$00000001)
    __rt_lib_init_alloca_1                   0x08000219   Thumb Code     0  libinit2.o(.ARM.Collect$$libinit$$0000002E)
    __rt_lib_init_argv_1                     0x08000219   Thumb Code     0  libinit2.o(.ARM.Collect$$libinit$$0000002C)
    __rt_lib_init_atexit_1                   0x08000219   Thumb Code     0  libinit2.o(.ARM.Collect$$libinit$$0000001B)
    __rt_lib_init_clock_1                    0x08000219   Thumb Code     0  libinit2.o(.ARM.Collect$$libinit$$00000021)
    __rt_lib_init_cpp_1                      0x08000219   Thumb Code     0  libinit2.o(.ARM.Collect$$libinit$$00000032)
    __rt_lib_init_exceptions_1               0x08000219   Thumb Code     0  libinit2.o(.ARM.Collect$$libinit$$00000030)
    __rt_lib_init_fp_trap_1                  0x08000219   Thumb Code     0  libinit2.o(.ARM.Collect$$libinit$$0000001F)
    __rt_lib_init_getenv_1                   0x08000219   Thumb Code     0  libinit2.o(.ARM.Collect$$libinit$$00000023)
    __rt_lib_init_heap_1                     0x08000219   Thumb Code     0  libinit2.o(.ARM.Collect$$libinit$$0000000A)
    __rt_lib_init_lc_collate_1               0x08000219   Thumb Code     0  libinit2.o(.ARM.Collect$$libinit$$00000011)
    __rt_lib_init_lc_ctype_1                 0x08000219   Thumb Code     0  libinit2.o(.ARM.Collect$$libinit$$00000013)
    __rt_lib_init_lc_monetary_1              0x08000219   Thumb Code     0  libinit2.o(.ARM.Collect$$libinit$$00000015)
    __rt_lib_init_lc_numeric_1               0x08000219   Thumb Code     0  libinit2.o(.ARM.Collect$$libinit$$00000017)
    __rt_lib_init_lc_time_1                  0x08000219   Thumb Code     0  libinit2.o(.ARM.Collect$$libinit$$00000019)
    __rt_lib_init_preinit_1                  0x08000219   Thumb Code     0  libinit2.o(.ARM.Collect$$libinit$$00000004)
    __rt_lib_init_rand_1                     0x08000219   Thumb Code     0  libinit2.o(.ARM.Collect$$libinit$$0000000E)
    __rt_lib_init_return                     0x08000219   Thumb Code     0  libinit2.o(.ARM.Collect$$libinit$$00000033)
    __rt_lib_init_signal_1                   0x08000219   Thumb Code     0  libinit2.o(.ARM.Collect$$libinit$$0000001D)
    __rt_lib_init_stdio_1                    0x08000219   Thumb Code     0  libinit2.o(.ARM.Collect$$libinit$$00000025)
    __rt_lib_init_user_alloc_1               0x08000219   Thumb Code     0  libinit2.o(.ARM.Collect$$libinit$$0000000C)
    __rt_lib_shutdown                        0x0800021b   Thumb Code     0  libshutdown.o(.ARM.Collect$$libshutdown$$00000000)
    __rt_lib_shutdown_cpp_1                  0x0800021d   Thumb Code     0  libshutdown2.o(.ARM.Collect$$libshutdown$$00000002)
    __rt_lib_shutdown_fp_trap_1              0x0800021d   Thumb Code     0  libshutdown2.o(.ARM.Collect$$libshutdown$$00000007)
    __rt_lib_shutdown_heap_1                 0x0800021d   Thumb Code     0  libshutdown2.o(.ARM.Collect$$libshutdown$$0000000F)
    __rt_lib_shutdown_return                 0x0800021d   Thumb Code     0  libshutdown2.o(.ARM.Collect$$libshutdown$$00000010)
    __rt_lib_shutdown_signal_1               0x0800021d   Thumb Code     0  libshutdown2.o(.ARM.Collect$$libshutdown$$0000000A)
    __rt_lib_shutdown_stdio_1                0x0800021d   Thumb Code     0  libshutdown2.o(.ARM.Collect$$libshutdown$$00000004)
    __rt_lib_shutdown_user_alloc_1           0x0800021d   Thumb Code     0  libshutdown2.o(.ARM.Collect$$libshutdown$$0000000C)
    __rt_entry                               0x0800021f   Thumb Code     0  __rtentry.o(.ARM.Collect$$rtentry$$00000000)
    __rt_entry_presh_1                       0x0800021f   Thumb Code     0  __rtentry2.o(.ARM.Collect$$rtentry$$00000002)
    __rt_entry_sh                            0x0800021f   Thumb Code     0  __rtentry4.o(.ARM.Collect$$rtentry$$00000004)
    __rt_entry_li                            0x08000225   Thumb Code     0  __rtentry2.o(.ARM.Collect$$rtentry$$0000000A)
    __rt_entry_postsh_1                      0x08000225   Thumb Code     0  __rtentry2.o(.ARM.Collect$$rtentry$$00000009)
    __rt_entry_main                          0x08000229   Thumb Code     0  __rtentry2.o(.ARM.Collect$$rtentry$$0000000D)
    __rt_entry_postli_1                      0x08000229   Thumb Code     0  __rtentry2.o(.ARM.Collect$$rtentry$$0000000C)
    __rt_exit                                0x08000231   Thumb Code     0  rtexit.o(.ARM.Collect$$rtexit$$00000000)
    __rt_exit_ls                             0x08000233   Thumb Code     0  rtexit2.o(.ARM.Collect$$rtexit$$00000003)
    __rt_exit_prels_1                        0x08000233   Thumb Code     0  rtexit2.o(.ARM.Collect$$rtexit$$00000002)
    __rt_exit_exit                           0x08000237   Thumb Code     0  rtexit2.o(.ARM.Collect$$rtexit$$00000004)
    Load_Drow_Dialog                         0x0800023d   Thumb Code    64  main.o(.text)
    lcd_draw_bline                           0x0800027d   Thumb Code   212  main.o(.text)
    ctp_test                                 0x08000351   Thumb Code   294  main.o(.text)
    main                                     0x08000477   Thumb Code   642  main.o(.text)
    NMI_Handler                              0x080006fd   Thumb Code     2  stm32f4xx_it.o(.text)
    HardFault_Handler                        0x080006ff   Thumb Code     4  stm32f4xx_it.o(.text)
    MemManage_Handler                        0x08000703   Thumb Code     4  stm32f4xx_it.o(.text)
    BusFault_Handler                         0x08000707   Thumb Code     4  stm32f4xx_it.o(.text)
    UsageFault_Handler                       0x0800070b   Thumb Code     4  stm32f4xx_it.o(.text)
    SVC_Handler                              0x0800070f   Thumb Code     2  stm32f4xx_it.o(.text)
    DebugMon_Handler                         0x08000711   Thumb Code     2  stm32f4xx_it.o(.text)
    PendSV_Handler                           0x08000713   Thumb Code     2  stm32f4xx_it.o(.text)
    SysTick_Handler                          0x08000715   Thumb Code     2  stm32f4xx_it.o(.text)
    SystemInit                               0x080007f5   Thumb Code    88  system_stm32f4xx.o(.text)
    SystemCoreClockUpdate                    0x0800084d   Thumb Code   174  system_stm32f4xx.o(.text)
    LED_Init                                 0x08000929   Thumb Code    60  led.o(.text)
    KEY_Init                                 0x08000969   Thumb Code    60  key.o(.text)
    Scan_Key                                 0x080009a5   Thumb Code   100  key.o(.text)
    Waiting_Key                              0x08000a09   Thumb Code    20  key.o(.text)
    WaitKey                                  0x08000a1d   Thumb Code    30  key.o(.text)
    WaitKeyBL                                0x08000a3b   Thumb Code    30  key.o(.text)
    Scan_Key_delay                           0x08000a59   Thumb Code    50  key.o(.text)
    Scan_FunctionKey                         0x08000a8b   Thumb Code   156  key.o(.text)
    KEY_Scan                                 0x08000b27   Thumb Code   188  key.o(.text)
    Delay_us                                 0x08000bf5   Thumb Code    30  if_port.o(.text)
    Delay_ms                                 0x08000c13   Thumb Code    32  if_port.o(.text)
    FSMC_IO_Init                             0x08000c33   Thumb Code   562  if_port.o(.text)
    FMSC_16_CmdWrite                         0x08000e65   Thumb Code     6  if_port.o(.text)
    FMSC_16_DataWrite                        0x08000e6b   Thumb Code     8  if_port.o(.text)
    FMSC_16_DataWrite_Pixel                  0x08000e73   Thumb Code     8  if_port.o(.text)
    FMSC_16_StatusRead                       0x08000e7b   Thumb Code    10  if_port.o(.text)
    FMSC_16_DataRead                         0x08000e85   Thumb Code    10  if_port.o(.text)
    LCD_CmdWrite                             0x08000e8f   Thumb Code    12  if_port.o(.text)
    LCD_DataWrite                            0x08000e9b   Thumb Code    12  if_port.o(.text)
    LCD_DataWrite_Pixel                      0x08000ea7   Thumb Code    12  if_port.o(.text)
    LCD_StatusRead                           0x08000eb3   Thumb Code    14  if_port.o(.text)
    LCD_DataRead                             0x08000ec1   Thumb Code    10  if_port.o(.text)
    Parallel_Init                            0x08000ecb   Thumb Code     8  if_port.o(.text)
    test_FSMCIO                              0x08000ed3   Thumb Code    38  if_port.o(.text)
    IIC_Init                                 0x08000f2d   Thumb Code    62  myiic.o(.text)
    IIC_Start                                0x08000f6b   Thumb Code    68  myiic.o(.text)
    IIC_Stop                                 0x08000faf   Thumb Code    62  myiic.o(.text)
    IIC_Wait_Ack                             0x08000fed   Thumb Code    82  myiic.o(.text)
    IIC_Ack                                  0x0800103f   Thumb Code    66  myiic.o(.text)
    IIC_NAck                                 0x08001081   Thumb Code    66  myiic.o(.text)
    IIC_Send_Byte                            0x080010c3   Thumb Code    90  myiic.o(.text)
    IIC_Read_Byte                            0x0800111d   Thumb Code    94  myiic.o(.text)
    AT24CXX_Init                             0x08001189   Thumb Code     8  24cxx.o(.text)
    AT24CXX_ReadOneByte                      0x08001191   Thumb Code    88  24cxx.o(.text)
    AT24CXX_WriteOneByte                     0x080011e9   Thumb Code    80  24cxx.o(.text)
    AT24CXX_WriteLenByte                     0x08001239   Thumb Code    42  24cxx.o(.text)
    AT24CXX_ReadLenByte                      0x08001263   Thumb Code    44  24cxx.o(.text)
    AT24CXX_Check                            0x0800128f   Thumb Code    46  24cxx.o(.text)
    AT24CXX_Read                             0x080012bd   Thumb Code    34  24cxx.o(.text)
    AT24CXX_Write                            0x080012df   Thumb Code    36  24cxx.o(.text)
    CT_Delay                                 0x08001305   Thumb Code    10  ctiic.o(.text)
    CT_IIC_Init                              0x0800130f   Thumb Code    60  ctiic.o(.text)
    CT_IIC_Start                             0x0800134b   Thumb Code    62  ctiic.o(.text)
    CT_IIC_Stop                              0x08001389   Thumb Code    56  ctiic.o(.text)
    CT_IIC_Wait_Ack                          0x080013c1   Thumb Code    78  ctiic.o(.text)
    CT_IIC_Ack                               0x0800140f   Thumb Code    66  ctiic.o(.text)
    CT_IIC_NAck                              0x08001451   Thumb Code    66  ctiic.o(.text)
    CT_IIC_Send_Byte                         0x08001493   Thumb Code    82  ctiic.o(.text)
    CT_IIC_Read_Byte                         0x080014e5   Thumb Code    92  ctiic.o(.text)
    TP_Write_Byte                            0x08001559   Thumb Code    64  touch.o(.text)
    TP_Read_AD                               0x08001599   Thumb Code   132  touch.o(.text)
    TP_Read_XOY                              0x0800161d   Thumb Code   120  touch.o(.text)
    TP_Read_XY                               0x08001695   Thumb Code    38  touch.o(.text)
    TP_Read_XY2                              0x080016bb   Thumb Code   192  touch.o(.text)
    TP_Drow_Touch_Point                      0x0800177b   Thumb Code    72  touch.o(.text)
    TP_Draw_Big_Point                        0x080017c3   Thumb Code    22  touch.o(.text)
    LCD_ShowChar                             0x080017d9   Thumb Code   278  touch.o(.text)
    LCD_Pow                                  0x080018ef   Thumb Code    22  touch.o(.text)
    LCD_ShowNum                              0x08001905   Thumb Code   188  touch.o(.text)
    TP_Scan                                  0x080019c1   Thumb Code   242  touch.o(.text)
    TP_Save_Adjdata                          0x08001ab3   Thumb Code   128  touch.o(.text)
    TP_Get_Adjdata                           0x08001b33   Thumb Code   170  touch.o(.text)
    TP_Adj_Info_Show                         0x08001bdd   Thumb Code   348  touch.o(.text)
    TP_Adjust                                0x08001d39   Thumb Code  1896  touch.o(.text)
    TP_Init                                  0x080024a1   Thumb Code   162  touch.o(.text)
    LCD_RegisterWrite                        0x08002599   Thumb Code    20  lt738.o(.text)
    LCD_RegisterRead                         0x080025ad   Thumb Code    20  lt738.o(.text)
    Check_Mem_WR_FIFO_not_Full               0x080025c1   Thumb Code    18  lt738.o(.text)
    Check_Mem_WR_FIFO_Empty                  0x080025d3   Thumb Code    18  lt738.o(.text)
    Check_Mem_RD_FIFO_not_Full               0x080025e5   Thumb Code    18  lt738.o(.text)
    Check_Mem_RD_FIFO_not_Empty              0x080025f7   Thumb Code    18  lt738.o(.text)
    Check_2D_Busy                            0x08002609   Thumb Code    18  lt738.o(.text)
    Check_SDRAM_Ready                        0x0800261b   Thumb Code    18  lt738.o(.text)
    Power_Saving_Status                      0x0800262d   Thumb Code    24  lt738.o(.text)
    Check_Power_is_Normal                    0x08002645   Thumb Code    18  lt738.o(.text)
    Check_Power_is_Saving                    0x08002657   Thumb Code    18  lt738.o(.text)
    Check_NO_Interrupt                       0x08002669   Thumb Code    18  lt738.o(.text)
    Check_Interrupt_Occur                    0x0800267b   Thumb Code    18  lt738.o(.text)
    Check_Busy_Draw                          0x0800268d   Thumb Code    18  lt738.o(.text)
    LT738_SW_Reset                           0x0800269f   Thumb Code    42  lt738.o(.text)
    Enable_PLL                               0x080026c9   Thumb Code    32  lt738.o(.text)
    LT738_Sleep                              0x080026e9   Thumb Code    26  lt738.o(.text)
    LT738_WakeUp                             0x08002703   Thumb Code    26  lt738.o(.text)
    Key_Scan_Enable                          0x0800271d   Thumb Code    26  lt738.o(.text)
    Key_Scan_Disable                         0x08002737   Thumb Code    26  lt738.o(.text)
    TFT_24bit                                0x08002751   Thumb Code    30  lt738.o(.text)
    TFT_18bit                                0x0800276f   Thumb Code    30  lt738.o(.text)
    TFT_16bit                                0x0800278d   Thumb Code    30  lt738.o(.text)
    TFT_LVDS                                 0x080027ab   Thumb Code    30  lt738.o(.text)
    LT738_I2CM_Enable                        0x080027c9   Thumb Code    26  lt738.o(.text)
    LT738_I2CM_Disable                       0x080027e3   Thumb Code    26  lt738.o(.text)
    Host_Bus_8bit                            0x080027fd   Thumb Code    26  lt738.o(.text)
    Host_Bus_16bit                           0x08002817   Thumb Code    26  lt738.o(.text)
    RGB_8b_8bpp                              0x08002831   Thumb Code    30  lt738.o(.text)
    RGB_8b_16bpp                             0x0800284f   Thumb Code    30  lt738.o(.text)
    RGB_8b_24bpp                             0x0800286d   Thumb Code    30  lt738.o(.text)
    RGB_16b_8bpp                             0x0800288b   Thumb Code    30  lt738.o(.text)
    RGB_16b_16bpp                            0x080028a9   Thumb Code    30  lt738.o(.text)
    RGB_16b_24bpp_mode1                      0x080028c7   Thumb Code    30  lt738.o(.text)
    RGB_16b_24bpp_mode2                      0x080028e5   Thumb Code    30  lt738.o(.text)
    MemRead_Left_Right_Top_Down              0x08002903   Thumb Code    30  lt738.o(.text)
    MemRead_Right_Left_Top_Down              0x08002921   Thumb Code    30  lt738.o(.text)
    MemRead_Top_Down_Left_Right              0x0800293f   Thumb Code    30  lt738.o(.text)
    MemRead_Down_Top_Left_Right              0x0800295d   Thumb Code    30  lt738.o(.text)
    MemWrite_Left_Right_Top_Down             0x0800297b   Thumb Code    30  lt738.o(.text)
    MemWrite_Right_Left_Top_Down             0x08002999   Thumb Code    30  lt738.o(.text)
    MemWrite_Top_Down_Left_Right             0x080029b7   Thumb Code    30  lt738.o(.text)
    MemWrite_Down_Top_Left_Right             0x080029d5   Thumb Code    30  lt738.o(.text)
    Interrupt_Active_Low                     0x080029f3   Thumb Code    26  lt738.o(.text)
    Interrupt_Active_High                    0x08002a0d   Thumb Code    26  lt738.o(.text)
    ExtInterrupt_Debounce                    0x08002a27   Thumb Code    26  lt738.o(.text)
    ExtInterrupt_Nodebounce                  0x08002a41   Thumb Code    26  lt738.o(.text)
    ExtInterrupt_Input_Low_Level_Trigger     0x08002a5b   Thumb Code    30  lt738.o(.text)
    ExtInterrupt_Input_High_Level_Trigger    0x08002a79   Thumb Code    30  lt738.o(.text)
    ExtInterrupt_Input_Falling_Edge_Trigger  0x08002a97   Thumb Code    30  lt738.o(.text)
    ExtInterrupt_Input_Rising_Edge_Trigger   0x08002ab5   Thumb Code    30  lt738.o(.text)
    LVDS_Format1                             0x08002ad3   Thumb Code    26  lt738.o(.text)
    LVDS_Format2                             0x08002aed   Thumb Code    26  lt738.o(.text)
    Graphic_Mode                             0x08002b07   Thumb Code    26  lt738.o(.text)
    Text_Mode                                0x08002b21   Thumb Code    26  lt738.o(.text)
    Memory_Select_SDRAM                      0x08002b3b   Thumb Code    30  lt738.o(.text)
    Memory_Select_Graphic_Cursor_RAM         0x08002b59   Thumb Code    30  lt738.o(.text)
    Memory_Select_Color_Palette_RAM          0x08002b77   Thumb Code    30  lt738.o(.text)
    Enable_Resume_Interrupt                  0x08002b95   Thumb Code    26  lt738.o(.text)
    Disable_Resume_Interrupt                 0x08002baf   Thumb Code    26  lt738.o(.text)
    Enable_ExtInterrupt_Input                0x08002bc9   Thumb Code    26  lt738.o(.text)
    Disable_ExtInterrupt_Input               0x08002be3   Thumb Code    26  lt738.o(.text)
    Enable_I2CM_Interrupt                    0x08002bfd   Thumb Code    26  lt738.o(.text)
    Disable_I2CM_Interrupt                   0x08002c17   Thumb Code    26  lt738.o(.text)
    Enable_Vsync_Interrupt                   0x08002c31   Thumb Code    26  lt738.o(.text)
    Disable_Vsync_Interrupt                  0x08002c4b   Thumb Code    26  lt738.o(.text)
    Enable_KeyScan_Interrupt                 0x08002c65   Thumb Code    26  lt738.o(.text)
    Disable_KeyScan_Interrupt                0x08002c7f   Thumb Code    26  lt738.o(.text)
    Enable_DMA_Draw_BTE_Interrupt            0x08002c99   Thumb Code    26  lt738.o(.text)
    Disable_DMA_Draw_BTE_Interrupt           0x08002cb3   Thumb Code    26  lt738.o(.text)
    Enable_PWM1_Interrupt                    0x08002ccd   Thumb Code    26  lt738.o(.text)
    Disable_PWM1_Interrupt                   0x08002ce7   Thumb Code    26  lt738.o(.text)
    Enable_PWM0_Interrupt                    0x08002d01   Thumb Code    26  lt738.o(.text)
    Disable_PWM0_Interrupt                   0x08002d1b   Thumb Code    26  lt738.o(.text)
    Read_Interrupt_status                    0x08002d35   Thumb Code    18  lt738.o(.text)
    Clear_Resume_Interrupt_Flag              0x08002d47   Thumb Code    26  lt738.o(.text)
    Clear_ExtInterrupt_Input_Flag            0x08002d61   Thumb Code    26  lt738.o(.text)
    Clear_I2CM_Interrupt_Flag                0x08002d7b   Thumb Code    26  lt738.o(.text)
    Clear_Vsync_Interrupt_Flag               0x08002d95   Thumb Code    26  lt738.o(.text)
    Clear_KeyScan_Interrupt_Flag             0x08002daf   Thumb Code    26  lt738.o(.text)
    Clear_Draw_BTE_Interrupt_Flag            0x08002dc9   Thumb Code    26  lt738.o(.text)
    Clear_PWM1_Interrupt_Flag                0x08002de3   Thumb Code    26  lt738.o(.text)
    Clear_PWM0_Interrupt_Flag                0x08002dfd   Thumb Code    26  lt738.o(.text)
    Mask_Resume_Interrupt_Flag               0x08002e17   Thumb Code    26  lt738.o(.text)
    Mask_ExtInterrupt_Input_Flag             0x08002e31   Thumb Code    26  lt738.o(.text)
    Mask_I2CM_Interrupt_Flag                 0x08002e4b   Thumb Code    26  lt738.o(.text)
    Mask_Vsync_Interrupt_Flag                0x08002e65   Thumb Code    26  lt738.o(.text)
    Mask_KeyScan_Interrupt_Flag              0x08002e7f   Thumb Code    26  lt738.o(.text)
    Mask_Draw_BTE_Interrupt_Flag             0x08002e99   Thumb Code    26  lt738.o(.text)
    Mask_PWM1_Interrupt_Flag                 0x08002eb3   Thumb Code    26  lt738.o(.text)
    Mask_PWM0_Interrupt_Flag                 0x08002ecd   Thumb Code    26  lt738.o(.text)
    Enable_Resume_Interrupt_Flag             0x08002ee7   Thumb Code    26  lt738.o(.text)
    Enable_ExtInterrupt_Inpur_Flag           0x08002f01   Thumb Code    26  lt738.o(.text)
    Enable_I2CM_Interrupt_Flag               0x08002f1b   Thumb Code    26  lt738.o(.text)
    Enable_Vsync_Interrupt_Flag              0x08002f35   Thumb Code    26  lt738.o(.text)
    Enable_KeyScan_Interrupt_Flag            0x08002f4f   Thumb Code    26  lt738.o(.text)
    Enable_Draw_BTE_Interrupt_Flag           0x08002f69   Thumb Code    26  lt738.o(.text)
    Enable_PWM1_Interrupt_Flag               0x08002f83   Thumb Code    26  lt738.o(.text)
    Enable_PWM0_Interrupt_Flag               0x08002f9d   Thumb Code    26  lt738.o(.text)
    Enable_GPIOF_PullUp                      0x08002fb7   Thumb Code    26  lt738.o(.text)
    Enable_GPIOE_PullUp                      0x08002fd1   Thumb Code    26  lt738.o(.text)
    Enable_GPIOD_PullUp                      0x08002feb   Thumb Code    26  lt738.o(.text)
    Enable_GPIOC_PullUp                      0x08003005   Thumb Code    26  lt738.o(.text)
    Enable_XDB15_8_PullUp                    0x0800301f   Thumb Code    26  lt738.o(.text)
    Enable_XDB7_0_PullUp                     0x08003039   Thumb Code    26  lt738.o(.text)
    Disable_GPIOF_PullUp                     0x08003053   Thumb Code    26  lt738.o(.text)
    Disable_GPIOE_PullUp                     0x0800306d   Thumb Code    26  lt738.o(.text)
    Disable_GPIOD_PullUp                     0x08003087   Thumb Code    26  lt738.o(.text)
    Disable_GPIOC_PullUp                     0x080030a1   Thumb Code    26  lt738.o(.text)
    Disable_XDB15_8_PullUp                   0x080030bb   Thumb Code    26  lt738.o(.text)
    Disable_XDB7_0_PullUp                    0x080030d5   Thumb Code    26  lt738.o(.text)
    XPDAT18_Set_GPIO_D7                      0x080030ef   Thumb Code    26  lt738.o(.text)
    XPDAT18_Set_KOUT4                        0x08003109   Thumb Code    26  lt738.o(.text)
    XPDAT17_Set_GPIO_D5                      0x08003123   Thumb Code    26  lt738.o(.text)
    XPDAT17_Set_KOUT2                        0x0800313d   Thumb Code    26  lt738.o(.text)
    XPDAT16_Set_GPIO_D4                      0x08003157   Thumb Code    26  lt738.o(.text)
    XPDAT16_Set_KOUT1                        0x08003171   Thumb Code    26  lt738.o(.text)
    XPDAT9_Set_GPIO_D3                       0x0800318b   Thumb Code    26  lt738.o(.text)
    XPDAT9_Set_KOUT3                         0x080031a5   Thumb Code    26  lt738.o(.text)
    XPDAT8_Set_GPIO_D2                       0x080031bf   Thumb Code    26  lt738.o(.text)
    XPDAT8_Set_KIN3                          0x080031d9   Thumb Code    26  lt738.o(.text)
    XPDAT2_Set_GPIO_D6                       0x080031f3   Thumb Code    26  lt738.o(.text)
    XPDAT2_Set_KIN4                          0x0800320d   Thumb Code    26  lt738.o(.text)
    XPDAT1_Set_GPIO_D1                       0x08003227   Thumb Code    26  lt738.o(.text)
    XPDAT1_Set_KIN2                          0x08003241   Thumb Code    26  lt738.o(.text)
    XPDAT0_Set_GPIO_D0                       0x0800325b   Thumb Code    26  lt738.o(.text)
    XPDAT0_Set_KIN1                          0x08003275   Thumb Code    26  lt738.o(.text)
    Enable_PIP1                              0x0800328f   Thumb Code    26  lt738.o(.text)
    Disable_PIP1                             0x080032a9   Thumb Code    26  lt738.o(.text)
    Enable_PIP2                              0x080032c3   Thumb Code    26  lt738.o(.text)
    Disable_PIP2                             0x080032dd   Thumb Code    26  lt738.o(.text)
    Select_PIP1_Parameter                    0x080032f7   Thumb Code    26  lt738.o(.text)
    Select_PIP2_Parameter                    0x08003311   Thumb Code    26  lt738.o(.text)
    Select_Main_Window_8bpp                  0x0800332b   Thumb Code    30  lt738.o(.text)
    Select_Main_Window_16bpp                 0x08003349   Thumb Code    30  lt738.o(.text)
    Select_Main_Window_24bpp                 0x08003367   Thumb Code    26  lt738.o(.text)
    Select_PIP2_Window_8bpp                  0x08003381   Thumb Code    30  lt738.o(.text)
    Select_PIP2_Window_16bpp                 0x0800339f   Thumb Code    30  lt738.o(.text)
    Select_PIP2_Window_24bpp                 0x080033bd   Thumb Code    30  lt738.o(.text)
    Select_PIP1_Window_8bpp                  0x080033db   Thumb Code    30  lt738.o(.text)
    Select_PIP1_Window_16bpp                 0x080033f9   Thumb Code    30  lt738.o(.text)
    Select_PIP1_Window_24bpp                 0x08003417   Thumb Code    30  lt738.o(.text)
    PCLK_Rising                              0x08003435   Thumb Code    26  lt738.o(.text)
    PCLK_Falling                             0x0800344f   Thumb Code    26  lt738.o(.text)
    Display_ON                               0x08003469   Thumb Code    26  lt738.o(.text)
    Display_OFF                              0x08003483   Thumb Code    26  lt738.o(.text)
    Color_Bar_ON                             0x0800349d   Thumb Code    26  lt738.o(.text)
    Color_Bar_OFF                            0x080034b7   Thumb Code    26  lt738.o(.text)
    HSCAN_L_to_R                             0x080034d1   Thumb Code    26  lt738.o(.text)
    HSCAN_R_to_L                             0x080034eb   Thumb Code    26  lt738.o(.text)
    VSCAN_T_to_B                             0x08003505   Thumb Code    26  lt738.o(.text)
    VSCAN_B_to_T                             0x0800351f   Thumb Code    26  lt738.o(.text)
    PDATA_Set_RGB                            0x08003539   Thumb Code    26  lt738.o(.text)
    PDATA_Set_RBG                            0x08003553   Thumb Code    30  lt738.o(.text)
    PDATA_Set_GRB                            0x08003571   Thumb Code    30  lt738.o(.text)
    PDATA_Set_GBR                            0x0800358f   Thumb Code    34  lt738.o(.text)
    PDATA_Set_BRG                            0x080035b1   Thumb Code    30  lt738.o(.text)
    PDATA_Set_BGR                            0x080035cf   Thumb Code    34  lt738.o(.text)
    PDATA_IDLE_STATE                         0x080035f1   Thumb Code    26  lt738.o(.text)
    HSYNC_Low_Active                         0x0800360b   Thumb Code    26  lt738.o(.text)
    HSYNC_High_Active                        0x08003625   Thumb Code    26  lt738.o(.text)
    VSYNC_Low_Active                         0x0800363f   Thumb Code    26  lt738.o(.text)
    VSYNC_High_Active                        0x08003659   Thumb Code    26  lt738.o(.text)
    DE_Low_Active                            0x08003673   Thumb Code    26  lt738.o(.text)
    DE_High_Active                           0x0800368d   Thumb Code    26  lt738.o(.text)
    Idle_DE_Low                              0x080036a7   Thumb Code    26  lt738.o(.text)
    Idle_DE_High                             0x080036c1   Thumb Code    26  lt738.o(.text)
    Idle_PCLK_Low                            0x080036db   Thumb Code    26  lt738.o(.text)
    Idle_PCLK_High                           0x080036f5   Thumb Code    26  lt738.o(.text)
    Idle_PDAT_Low                            0x0800370f   Thumb Code    26  lt738.o(.text)
    Idle_PDAT_High                           0x08003729   Thumb Code    26  lt738.o(.text)
    Idle_HSYNC_Low                           0x08003743   Thumb Code    26  lt738.o(.text)
    Idle_HSYNC_High                          0x0800375d   Thumb Code    26  lt738.o(.text)
    Idle_VSYNC_Low                           0x08003777   Thumb Code    26  lt738.o(.text)
    Idle_VSYNC_High                          0x08003791   Thumb Code    26  lt738.o(.text)
    LCD_HorizontalWidth_VerticalHeight       0x080037ab   Thumb Code   160  lt738.o(.text)
    LCD_Horizontal_Non_Display               0x0800384b   Thumb Code    90  lt738.o(.text)
    LCD_HSYNC_Start_Position                 0x080038a5   Thumb Code    50  lt738.o(.text)
    LCD_HSYNC_Pulse_Width                    0x080038d7   Thumb Code    50  lt738.o(.text)
    LCD_Vertical_Non_Display                 0x08003909   Thumb Code    34  lt738.o(.text)
    LCD_VSYNC_Start_Position                 0x0800392b   Thumb Code    22  lt738.o(.text)
    LCD_VSYNC_Pulse_Width                    0x08003941   Thumb Code    22  lt738.o(.text)
    Main_Image_Start_Address                 0x08003957   Thumb Code    42  lt738.o(.text)
    Main_Image_Width                         0x08003981   Thumb Code    22  lt738.o(.text)
    Main_Window_Start_XY                     0x08003997   Thumb Code    40  lt738.o(.text)
    PIP_Display_Start_XY                     0x080039bf   Thumb Code    40  lt738.o(.text)
    PIP_Image_Start_Address                  0x080039e7   Thumb Code    42  lt738.o(.text)
    PIP_Image_Width                          0x08003a11   Thumb Code    22  lt738.o(.text)
    PIP_Window_Image_Start_XY                0x08003a27   Thumb Code    40  lt738.o(.text)
    PIP_Window_Width_Height                  0x08003a4f   Thumb Code    40  lt738.o(.text)
    Enable_Graphic_Cursor                    0x08003a77   Thumb Code    26  lt738.o(.text)
    Disable_Graphic_Cursor                   0x08003a91   Thumb Code    26  lt738.o(.text)
    Select_Graphic_Cursor_1                  0x08003aab   Thumb Code    30  lt738.o(.text)
    Select_Graphic_Cursor_2                  0x08003ac9   Thumb Code    30  lt738.o(.text)
    Select_Graphic_Cursor_3                  0x08003ae7   Thumb Code    30  lt738.o(.text)
    Select_Graphic_Cursor_4                  0x08003b05   Thumb Code    30  lt738.o(.text)
    Enable_Text_Cursor                       0x08003b23   Thumb Code    26  lt738.o(.text)
    Disable_Text_Cursor                      0x08003b3d   Thumb Code    26  lt738.o(.text)
    Enable_Text_Cursor_Blinking              0x08003b57   Thumb Code    26  lt738.o(.text)
    Disable_Text_Cursor_Blinking             0x08003b71   Thumb Code    26  lt738.o(.text)
    Blinking_Time_Frames                     0x08003b8b   Thumb Code    18  lt738.o(.text)
    Text_Cursor_H_V                          0x08003b9d   Thumb Code    32  lt738.o(.text)
    Graphic_Cursor_XY                        0x08003bbd   Thumb Code    40  lt738.o(.text)
    Set_Graphic_Cursor_Color_1               0x08003be5   Thumb Code    14  lt738.o(.text)
    Set_Graphic_Cursor_Color_2               0x08003bf3   Thumb Code    14  lt738.o(.text)
    Canvas_Image_Start_address               0x08003c01   Thumb Code    42  lt738.o(.text)
    Canvas_image_width                       0x08003c2b   Thumb Code    22  lt738.o(.text)
    Active_Window_XY                         0x08003c41   Thumb Code    40  lt738.o(.text)
    Active_Window_WH                         0x08003c69   Thumb Code    40  lt738.o(.text)
    Select_Write_Data_Position               0x08003c91   Thumb Code    26  lt738.o(.text)
    Select_Read_Data_Position                0x08003cab   Thumb Code    26  lt738.o(.text)
    Memory_XY_Mode                           0x08003cc5   Thumb Code    26  lt738.o(.text)
    Memory_Linear_Mode                       0x08003cdf   Thumb Code    26  lt738.o(.text)
    Memory_8bpp_Mode                         0x08003cf9   Thumb Code    30  lt738.o(.text)
    Memory_16bpp_Mode                        0x08003d17   Thumb Code    30  lt738.o(.text)
    Memory_24bpp_Mode                        0x08003d35   Thumb Code    30  lt738.o(.text)
    Goto_Pixel_XY                            0x08003d53   Thumb Code    40  lt738.o(.text)
    Goto_Linear_Addr                         0x08003d7b   Thumb Code    42  lt738.o(.text)
    Goto_Text_XY                             0x08003da5   Thumb Code    40  lt738.o(.text)
    Start_Line                               0x08003dcd   Thumb Code    20  lt738.o(.text)
    Start_Triangle                           0x08003de1   Thumb Code    20  lt738.o(.text)
    Start_Triangle_Fill                      0x08003df5   Thumb Code    20  lt738.o(.text)
    Line_Start_XY                            0x08003e09   Thumb Code    56  lt738.o(.text)
    Line_End_XY                              0x08003e41   Thumb Code    56  lt738.o(.text)
    Triangle_Point1_XY                       0x08003e79   Thumb Code    56  lt738.o(.text)
    Triangle_Point2_XY                       0x08003eb1   Thumb Code    56  lt738.o(.text)
    Triangle_Point3_XY                       0x08003ee9   Thumb Code    56  lt738.o(.text)
    Square_Start_XY                          0x08003f21   Thumb Code    56  lt738.o(.text)
    Square_End_XY                            0x08003f59   Thumb Code    56  lt738.o(.text)
    Start_Circle_or_Ellipse                  0x08003f91   Thumb Code    20  lt738.o(.text)
    Start_Circle_or_Ellipse_Fill             0x08003fa5   Thumb Code    20  lt738.o(.text)
    Start_Left_Down_Curve                    0x08003fb9   Thumb Code    20  lt738.o(.text)
    Start_Left_Up_Curve                      0x08003fcd   Thumb Code    20  lt738.o(.text)
    Start_Right_Up_Curve                     0x08003fe1   Thumb Code    20  lt738.o(.text)
    Start_Right_Down_Curve                   0x08003ff5   Thumb Code    20  lt738.o(.text)
    Start_Left_Down_Curve_Fill               0x08004009   Thumb Code    20  lt738.o(.text)
    Start_Left_Up_Curve_Fill                 0x0800401d   Thumb Code    20  lt738.o(.text)
    Start_Right_Up_Curve_Fill                0x08004031   Thumb Code    20  lt738.o(.text)
    Start_Right_Down_Curve_Fill              0x08004045   Thumb Code    20  lt738.o(.text)
    Start_Square                             0x08004059   Thumb Code    20  lt738.o(.text)
    Start_Square_Fill                        0x0800406d   Thumb Code    20  lt738.o(.text)
    Start_Circle_Square                      0x08004081   Thumb Code    20  lt738.o(.text)
    Start_Circle_Square_Fill                 0x08004095   Thumb Code    20  lt738.o(.text)
    Circle_Center_XY                         0x080040a9   Thumb Code    56  lt738.o(.text)
    Ellipse_Center_XY                        0x080040e1   Thumb Code    56  lt738.o(.text)
    Circle_Radius_R                          0x08004119   Thumb Code    54  lt738.o(.text)
    Ellipse_Radius_RxRy                      0x0800414f   Thumb Code    56  lt738.o(.text)
    Circle_Square_Radius_RxRy                0x08004187   Thumb Code    56  lt738.o(.text)
    Set_PWM_Prescaler_1_to_256               0x080041bf   Thumb Code    22  lt738.o(.text)
    Select_PWM1_Clock_Divided_By_1           0x080041d5   Thumb Code    30  lt738.o(.text)
    Select_PWM1_Clock_Divided_By_2           0x080041f3   Thumb Code    30  lt738.o(.text)
    Select_PWM1_Clock_Divided_By_4           0x08004211   Thumb Code    30  lt738.o(.text)
    Select_PWM1_Clock_Divided_By_8           0x0800422f   Thumb Code    30  lt738.o(.text)
    Select_PWM0_Clock_Divided_By_1           0x0800424d   Thumb Code    30  lt738.o(.text)
    Select_PWM0_Clock_Divided_By_2           0x0800426b   Thumb Code    30  lt738.o(.text)
    Select_PWM0_Clock_Divided_By_4           0x08004289   Thumb Code    30  lt738.o(.text)
    Select_PWM0_Clock_Divided_By_8           0x080042a7   Thumb Code    30  lt738.o(.text)
    Select_PWM1_is_ErrorFlag                 0x080042c5   Thumb Code    26  lt738.o(.text)
    Select_PWM1                              0x080042df   Thumb Code    30  lt738.o(.text)
    Select_PWM1_is_Osc_Clock                 0x080042fd   Thumb Code    30  lt738.o(.text)
    Select_PWM0_is_GPIO_C7                   0x0800431b   Thumb Code    26  lt738.o(.text)
    Select_PWM0                              0x08004335   Thumb Code    30  lt738.o(.text)
    Select_PWM0_is_Core_Clock                0x08004353   Thumb Code    30  lt738.o(.text)
    Enable_PWM1_Inverter                     0x08004371   Thumb Code    26  lt738.o(.text)
    Disable_PWM1_Inverter                    0x0800438b   Thumb Code    26  lt738.o(.text)
    Auto_Reload_PWM1                         0x080043a5   Thumb Code    26  lt738.o(.text)
    One_Shot_PWM1                            0x080043bf   Thumb Code    26  lt738.o(.text)
    Start_PWM1                               0x080043d9   Thumb Code    26  lt738.o(.text)
    Stop_PWM1                                0x080043f3   Thumb Code    26  lt738.o(.text)
    Enable_PWM0_Dead_Zone                    0x0800440d   Thumb Code    26  lt738.o(.text)
    Disable_PWM0_Dead_Zone                   0x08004427   Thumb Code    26  lt738.o(.text)
    Enable_PWM0_Inverter                     0x08004441   Thumb Code    26  lt738.o(.text)
    Disable_PWM0_Inverter                    0x0800445b   Thumb Code    26  lt738.o(.text)
    Auto_Reload_PWM0                         0x08004475   Thumb Code    26  lt738.o(.text)
    One_Shot_PWM0                            0x0800448f   Thumb Code    26  lt738.o(.text)
    Start_PWM0                               0x080044a9   Thumb Code    26  lt738.o(.text)
    Stop_PWM0                                0x080044c3   Thumb Code    26  lt738.o(.text)
    Set_Timer0_Dead_Zone_Length              0x080044dd   Thumb Code    18  lt738.o(.text)
    Set_Timer0_Compare_Buffer                0x080044ef   Thumb Code    30  lt738.o(.text)
    Set_Timer0_Count_Buffer                  0x0800450d   Thumb Code    30  lt738.o(.text)
    Set_Timer1_Compare_Buffer                0x0800452b   Thumb Code    30  lt738.o(.text)
    Set_Timer1_Count_Buffer                  0x08004549   Thumb Code    30  lt738.o(.text)
    BTE_Enable                               0x08004567   Thumb Code    26  lt738.o(.text)
    BTE_Disable                              0x08004581   Thumb Code    26  lt738.o(.text)
    Check_BTE_Busy                           0x0800459b   Thumb Code    18  lt738.o(.text)
    Pattern_Format_8X8                       0x080045ad   Thumb Code    26  lt738.o(.text)
    Pattern_Format_16X16                     0x080045c7   Thumb Code    26  lt738.o(.text)
    BTE_ROP_Code                             0x080045e1   Thumb Code    34  lt738.o(.text)
    BTE_Operation_Code                       0x08004603   Thumb Code    30  lt738.o(.text)
    BTE_S0_Color_8bpp                        0x08004621   Thumb Code    30  lt738.o(.text)
    BTE_S0_Color_16bpp                       0x0800463f   Thumb Code    30  lt738.o(.text)
    BTE_S0_Color_24bpp                       0x0800465d   Thumb Code    26  lt738.o(.text)
    BTE_S1_Color_8bpp                        0x08004677   Thumb Code    34  lt738.o(.text)
    BTE_S1_Color_16bpp                       0x08004699   Thumb Code    34  lt738.o(.text)
    BTE_S1_Color_24bpp                       0x080046bb   Thumb Code    34  lt738.o(.text)
    BTE_S1_Color_Constant                    0x080046dd   Thumb Code    34  lt738.o(.text)
    BTE_S1_Color_8bit_Alpha                  0x080046ff   Thumb Code    34  lt738.o(.text)
    BTE_S1_Color_16bit_Alpha                 0x08004721   Thumb Code    34  lt738.o(.text)
    BTE_Destination_Color_8bpp               0x08004743   Thumb Code    30  lt738.o(.text)
    BTE_Destination_Color_16bpp              0x08004761   Thumb Code    30  lt738.o(.text)
    BTE_Destination_Color_24bpp              0x0800477f   Thumb Code    26  lt738.o(.text)
    BTE_S0_Memory_Start_Address              0x08004799   Thumb Code    42  lt738.o(.text)
    BTE_S0_Image_Width                       0x080047c3   Thumb Code    22  lt738.o(.text)
    BTE_S0_Window_Start_XY                   0x080047d9   Thumb Code    40  lt738.o(.text)
    BTE_S1_Memory_Start_Address              0x08004801   Thumb Code    42  lt738.o(.text)
    S1_Constant_color_256                    0x0800482b   Thumb Code    46  lt738.o(.text)
    S1_Constant_color_65k                    0x08004859   Thumb Code    46  lt738.o(.text)
    S1_Constant_color_16M                    0x08004887   Thumb Code    46  lt738.o(.text)
    BTE_S1_Image_Width                       0x080048b5   Thumb Code    22  lt738.o(.text)
    BTE_S1_Window_Start_XY                   0x080048cb   Thumb Code    40  lt738.o(.text)
    BTE_Destination_Memory_Start_Address     0x080048f3   Thumb Code    42  lt738.o(.text)
    BTE_Destination_Image_Width              0x0800491d   Thumb Code    22  lt738.o(.text)
    BTE_Destination_Window_Start_XY          0x08004933   Thumb Code    40  lt738.o(.text)
    BTE_Window_Size                          0x0800495b   Thumb Code    40  lt738.o(.text)
    BTE_Alpha_Blending_Effect                0x08004983   Thumb Code    18  lt738.o(.text)
    Font_Select_UserDefine_Mode              0x08004995   Thumb Code    30  lt738.o(.text)
    CGROM_Select_Internal_CGROM              0x080049b3   Thumb Code    30  lt738.o(.text)
    CGROM_Select_Genitop_FontROM             0x080049d1   Thumb Code    30  lt738.o(.text)
    Font_Select_8x16_16x16                   0x080049ef   Thumb Code    30  lt738.o(.text)
    Font_Select_12x24_24x24                  0x08004a0d   Thumb Code    30  lt738.o(.text)
    Font_Select_16x32_32x32                  0x08004a2b   Thumb Code    30  lt738.o(.text)
    Internal_CGROM_Select_ISOIEC8859_1       0x08004a49   Thumb Code    30  lt738.o(.text)
    Internal_CGROM_Select_ISOIEC8859_2       0x08004a67   Thumb Code    30  lt738.o(.text)
    Internal_CGROM_Select_ISOIEC8859_3       0x08004a85   Thumb Code    30  lt738.o(.text)
    Internal_CGROM_Select_ISOIEC8859_4       0x08004aa3   Thumb Code    30  lt738.o(.text)
    Enable_Font_Alignment                    0x08004ac1   Thumb Code    26  lt738.o(.text)
    Disable_Font_Alignment                   0x08004adb   Thumb Code    26  lt738.o(.text)
    Font_Background_select_Transparency      0x08004af5   Thumb Code    26  lt738.o(.text)
    Font_Background_select_Color             0x08004b0f   Thumb Code    26  lt738.o(.text)
    Font_0_degree                            0x08004b29   Thumb Code    26  lt738.o(.text)
    Font_90_degree                           0x08004b43   Thumb Code    26  lt738.o(.text)
    Font_Width_X1                            0x08004b5d   Thumb Code    30  lt738.o(.text)
    Font_Width_X2                            0x08004b7b   Thumb Code    30  lt738.o(.text)
    Font_Width_X3                            0x08004b99   Thumb Code    30  lt738.o(.text)
    Font_Width_X4                            0x08004bb7   Thumb Code    30  lt738.o(.text)
    Font_Height_X1                           0x08004bd5   Thumb Code    30  lt738.o(.text)
    Font_Height_X2                           0x08004bf3   Thumb Code    30  lt738.o(.text)
    Font_Height_X3                           0x08004c11   Thumb Code    30  lt738.o(.text)
    Font_Height_X4                           0x08004c2f   Thumb Code    30  lt738.o(.text)
    GTFont_Select_GT21L16TW_GT21H16T1W       0x08004c4d   Thumb Code    34  lt738.o(.text)
    GTFont_Select_GT23L16U2W                 0x08004c6f   Thumb Code    34  lt738.o(.text)
    GTFont_Select_GT23L24T3Y_GT23H24T3Y      0x08004c91   Thumb Code    34  lt738.o(.text)
    GTFont_Select_GT23L24M1Z                 0x08004cb3   Thumb Code    34  lt738.o(.text)
    GTFont_Select_GT23L32S4W_GT23H32S4W      0x08004cd5   Thumb Code    34  lt738.o(.text)
    GTFont_Select_GT20L24F6Y                 0x08004cf7   Thumb Code    34  lt738.o(.text)
    GTFont_Select_GT21L24S1W                 0x08004d19   Thumb Code    34  lt738.o(.text)
    GTFont_Select_GT22L16A1Y                 0x08004d3b   Thumb Code    34  lt738.o(.text)
    Set_GTFont_Decoder                       0x08004d5d   Thumb Code    18  lt738.o(.text)
    Font_Line_Distance                       0x08004d6f   Thumb Code    18  lt738.o(.text)
    Set_Font_to_Font_Width                   0x08004d81   Thumb Code    18  lt738.o(.text)
    Foreground_RGB                           0x08004d93   Thumb Code    46  lt738.o(.text)
    Foreground_color_256                     0x08004dc1   Thumb Code    46  lt738.o(.text)
    Foreground_color_65k                     0x08004def   Thumb Code    46  lt738.o(.text)
    Foreground_color_16M                     0x08004e1d   Thumb Code    46  lt738.o(.text)
    Background_RGB                           0x08004e4b   Thumb Code    46  lt738.o(.text)
    Background_color_256                     0x08004e79   Thumb Code    46  lt738.o(.text)
    Background_color_65k                     0x08004ea7   Thumb Code    46  lt738.o(.text)
    Background_color_16M                     0x08004ed5   Thumb Code    46  lt738.o(.text)
    CGRAM_Start_address                      0x08004f03   Thumb Code    58  lt738.o(.text)
    Power_Normal_Mode                        0x08004f3d   Thumb Code    16  lt738.o(.text)
    Power_Saving_Standby_Mode                0x08004f4d   Thumb Code    28  lt738.o(.text)
    Power_Saving_Suspend_Mode                0x08004f69   Thumb Code    16  lt738.o(.text)
    Power_Saving_Sleep_Mode                  0x08004f79   Thumb Code    16  lt738.o(.text)
    LT738_I2CM_Clock_Prescale                0x08004f89   Thumb Code    30  lt738.o(.text)
    LT738_I2CM_Transmit_Data                 0x08004fa7   Thumb Code    18  lt738.o(.text)
    LT738_I2CM_Receiver_Data                 0x08004fb9   Thumb Code    18  lt738.o(.text)
    LT738_I2CM_Stop                          0x08004fcb   Thumb Code    16  lt738.o(.text)
    LT738_I2CM_Read_With_Ack                 0x08004fdb   Thumb Code    16  lt738.o(.text)
    LT738_I2CM_Read_With_Nack                0x08004feb   Thumb Code    16  lt738.o(.text)
    LT738_I2CM_Write_With_Start              0x08004ffb   Thumb Code    16  lt738.o(.text)
    LT738_I2CM_Write                         0x0800500b   Thumb Code    16  lt738.o(.text)
    LT738_I2CM_Check_Slave_ACK               0x0800501b   Thumb Code    30  lt738.o(.text)
    LT738_I2CM_Bus_Busy                      0x08005039   Thumb Code    30  lt738.o(.text)
    LT738_I2CM_transmit_Progress             0x08005057   Thumb Code    30  lt738.o(.text)
    LT738_I2CM_Arbitration                   0x08005075   Thumb Code    22  lt738.o(.text)
    Set_GPIO_A_In_Out                        0x0800508b   Thumb Code    18  lt738.o(.text)
    Write_GPIO_A_7_0                         0x0800509d   Thumb Code    18  lt738.o(.text)
    Read_GPIO_A_7_0                          0x080050af   Thumb Code    18  lt738.o(.text)
    Write_GPIO_B_7_4                         0x080050c1   Thumb Code    18  lt738.o(.text)
    Read_GPIO_B_7_0                          0x080050d3   Thumb Code    18  lt738.o(.text)
    Set_GPIO_C_In_Out                        0x080050e5   Thumb Code    18  lt738.o(.text)
    Write_GPIO_C_7_0                         0x080050f7   Thumb Code    18  lt738.o(.text)
    Read_GPIO_C_7_0                          0x08005109   Thumb Code    18  lt738.o(.text)
    Set_GPIO_D_In_Out                        0x0800511b   Thumb Code    18  lt738.o(.text)
    Write_GPIO_D_7_0                         0x0800512d   Thumb Code    18  lt738.o(.text)
    Read_GPIO_D_7_0                          0x0800513f   Thumb Code    18  lt738.o(.text)
    Set_GPIO_E_In_Out                        0x08005151   Thumb Code    18  lt738.o(.text)
    Write_GPIO_E_7_0                         0x08005163   Thumb Code    18  lt738.o(.text)
    Read_GPIO_E_7_0                          0x08005175   Thumb Code    18  lt738.o(.text)
    Set_GPIO_F_In_Out                        0x08005187   Thumb Code    18  lt738.o(.text)
    Write_GPIO_F_7_0                         0x08005199   Thumb Code    18  lt738.o(.text)
    Read_GPIO_F_7_0                          0x080051ab   Thumb Code    18  lt738.o(.text)
    Long_Key_enable                          0x080051bd   Thumb Code    26  lt738.o(.text)
    Key_Scan_Freg                            0x080051d7   Thumb Code    34  lt738.o(.text)
    Key_Scan_Wakeup_Function_Enable          0x080051f9   Thumb Code    26  lt738.o(.text)
    Long_Key_Timing_Adjustment               0x08005213   Thumb Code    30  lt738.o(.text)
    Numbers_of_Key_Hit                       0x08005231   Thumb Code    22  lt738.o(.text)
    Read_Key_Strobe_Data_0                   0x08005247   Thumb Code    18  lt738.o(.text)
    Read_Key_Strobe_Data_1                   0x08005259   Thumb Code    18  lt738.o(.text)
    Read_Key_Strobe_Data_2                   0x0800526b   Thumb Code    18  lt738.o(.text)
    Show_String                              0x0800527d   Thumb Code    44  lt738.o(.text)
    Show_picture                             0x080052a9   Thumb Code    36  lt738.o(.text)
    Display_picture                          0x080052cd   Thumb Code   152  lt738_demo.o(.text)
    GRAY_32                                  0x08005365   Thumb Code    56  lt738_demo.o(.text)
    WB_block                                 0x0800539d   Thumb Code   324  lt738_demo.o(.text)
    Show                                     0x080054e1   Thumb Code   142  lt738_demo.o(.text)
    LT738_HW_Reset                           0x08005571   Thumb Code    98  lt738_lib.o(.text)
    System_Check_Temp                        0x080055d3   Thumb Code   108  lt738_lib.o(.text)
    LT738_PLL_Initial                        0x0800563f   Thumb Code   278  lt738_lib.o(.text)
    LT738_SDRAM_initail                      0x08005755   Thumb Code    78  lt738_lib.o(.text)
    Set_LCD_Panel                            0x080057a3   Thumb Code   108  lt738_lib.o(.text)
    LT738_initial                            0x0800580f   Thumb Code    20  lt738_lib.o(.text)
    LT738_Init                               0x08005823   Thumb Code    56  lt738_lib.o(.text)
    MPU8_8bpp_Memory_Write                   0x0800585b   Thumb Code    98  lt738_lib.o(.text)
    MPU8_16bpp_Memory_Write                  0x080058bd   Thumb Code   110  lt738_lib.o(.text)
    MPU8_24bpp_Memory_Write                  0x0800592b   Thumb Code   154  lt738_lib.o(.text)
    MPU16_16bpp_Memory_Write                 0x080059c5   Thumb Code    98  lt738_lib.o(.text)
    MPU16_24bpp_Mode1_Memory_Write           0x08005a27   Thumb Code   128  lt738_lib.o(.text)
    MPU16_24bpp_Mode2_Memory_Write           0x08005aa7   Thumb Code   110  lt738_lib.o(.text)
    LT738_DrawLine                           0x08005b15   Thumb Code    52  lt738_lib.o(.text)
    LT738_DrawLine_Width                     0x08005b49   Thumb Code   246  lt738_lib.o(.text)
    LT738_DrawCircle                         0x08005c3f   Thumb Code    44  lt738_lib.o(.text)
    LT738_DrawCircle_Fill                    0x08005c6b   Thumb Code    44  lt738_lib.o(.text)
    LT738_DrawCircle_Width                   0x08005c97   Thumb Code    48  lt738_lib.o(.text)
    LT738_DrawEllipse                        0x08005cc7   Thumb Code    52  lt738_lib.o(.text)
    LT738_DrawEllipse_Fill                   0x08005cfb   Thumb Code    52  lt738_lib.o(.text)
    LT738_DrawEllipse_Width                  0x08005d2f   Thumb Code    58  lt738_lib.o(.text)
    LT738_DrawSquare                         0x08005d69   Thumb Code    52  lt738_lib.o(.text)
    LT738_DrawSquare_Fill                    0x08005d9d   Thumb Code    52  lt738_lib.o(.text)
    LT738_DrawSquare_Width                   0x08005dd1   Thumb Code    78  lt738_lib.o(.text)
    LT738_DrawCircleSquare                   0x08005e1f   Thumb Code    64  lt738_lib.o(.text)
    LT738_DrawCircleSquare_Fill              0x08005e5f   Thumb Code    64  lt738_lib.o(.text)
    LT738_DrawCircleSquare_Width             0x08005e9f   Thumb Code    86  lt738_lib.o(.text)
    LT738_DrawTriangle                       0x08005ef5   Thumb Code    64  lt738_lib.o(.text)
    LT738_DrawTriangle_Fill                  0x08005f35   Thumb Code   100  lt738_lib.o(.text)
    LT738_DrawTriangle_Frame                 0x08005f99   Thumb Code    54  lt738_lib.o(.text)
    LT738_DrawLeftUpCurve                    0x08005fcf   Thumb Code    52  lt738_lib.o(.text)
    LT738_DrawLeftDownCurve                  0x08006003   Thumb Code    52  lt738_lib.o(.text)
    LT738_DrawRightUpCurve                   0x08006037   Thumb Code    52  lt738_lib.o(.text)
    LT738_DrawRightDownCurve                 0x0800606b   Thumb Code    52  lt738_lib.o(.text)
    LT738_SelectDrawCurve                    0x0800609f   Thumb Code   114  lt738_lib.o(.text)
    LT738_DrawLeftUpCurve_Fill               0x08006111   Thumb Code    52  lt738_lib.o(.text)
    LT738_DrawLeftDownCurve_Fill             0x08006145   Thumb Code    52  lt738_lib.o(.text)
    LT738_DrawRightUpCurve_Fill              0x08006179   Thumb Code    52  lt738_lib.o(.text)
    LT738_DrawRightDownCurve_Fill            0x080061ad   Thumb Code    52  lt738_lib.o(.text)
    LT738_SelectDrawCurve_Fill               0x080061e1   Thumb Code   114  lt738_lib.o(.text)
    LT738_DrawQuadrilateral                  0x08006253   Thumb Code    88  lt738_lib.o(.text)
    LT738_DrawQuadrilateral_Fill             0x080062ab   Thumb Code    88  lt738_lib.o(.text)
    LT738_DrawPentagon                       0x08006303   Thumb Code    92  lt738_lib.o(.text)
    LT738_DrawPentagon_Fill                  0x0800635f   Thumb Code    92  lt738_lib.o(.text)
    LT738_DrawCylinder                       0x080063bb   Thumb Code   166  lt738_lib.o(.text)
    LT738_DrawQuadrangular                   0x08006461   Thumb Code   130  lt738_lib.o(.text)
    LT738_MakeTable                          0x080064e3   Thumb Code   194  lt738_lib.o(.text)
    LT738_Color_Bar_ON                       0x080065a5   Thumb Code     8  lt738_lib.o(.text)
    LT738_Color_Bar_OFF                      0x080065ad   Thumb Code     8  lt738_lib.o(.text)
    LT738_Select_Internal_Font_Init          0x080065b5   Thumb Code   142  lt738_lib.o(.text)
    LT738_Print_Internal_Font_String         0x08006643   Thumb Code    54  lt738_lib.o(.text)
    LT738_Print_Outside_Font_String          0x08006679   Thumb Code   166  lt738_lib.o(.text)
    LT738_BTE_Memory_Copy_ColorExpansion_8   0x0800671f   Thumb Code   116  lt738_lib.o(.text)
    LT738_BTE_Memory_Copy_ColorExpansion_Chroma_key_8 0x08006793   Thumb Code   112  lt738_lib.o(.text)
    LT738_Text_cursor_Init                   0x08006803   Thumb Code    48  lt738_lib.o(.text)
    LT738_Enable_Text_Cursor                 0x08006833   Thumb Code     8  lt738_lib.o(.text)
    LT738_Disable_Text_Cursor                0x0800683b   Thumb Code     8  lt738_lib.o(.text)
    LT738_Graphic_cursor_Init                0x08006843   Thumb Code   126  lt738_lib.o(.text)
    LT738_Set_Graphic_cursor_Pos             0x080068c1   Thumb Code    64  lt738_lib.o(.text)
    LT738_Enable_Graphic_Cursor              0x08006901   Thumb Code     8  lt738_lib.o(.text)
    LT738_Disable_Graphic_Cursor             0x08006909   Thumb Code     8  lt738_lib.o(.text)
    LT738_PIP_Init                           0x08006911   Thumb Code   124  lt738_lib.o(.text)
    LT738_Set_DisWindowPos                   0x0800698d   Thumb Code    78  lt738_lib.o(.text)
    BTE_Solid_Fill                           0x080069db   Thumb Code    76  lt738_lib.o(.text)
    LT738_BTE_Memory_Copy                    0x08006a27   Thumb Code   130  lt738_lib.o(.text)
    LT738_BTE_Memory_Copy_Chroma_key         0x08006aa9   Thumb Code   106  lt738_lib.o(.text)
    LT738_BTE_Pattern_Fill                   0x08006b13   Thumb Code   116  lt738_lib.o(.text)
    LT738_BTE_Pattern_Fill_With_Chroma_key   0x08006b87   Thumb Code   128  lt738_lib.o(.text)
    LT738_BTE_MCU_Write_MCU_16bit            0x08006c07   Thumb Code   164  lt738_lib.o(.text)
    LT738_BTE_MCU_Write_Chroma_key_MCU_16bit 0x08006cab   Thumb Code   132  lt738_lib.o(.text)
    LT738_BTE_MCU_Write_ColorExpansion_MCU_16bit 0x08006d2f   Thumb Code   164  lt738_lib.o(.text)
    LT738_BTE_MCU_Write_ColorExpansion_Chroma_key_MCU_16bit 0x08006dd3   Thumb Code   156  lt738_lib.o(.text)
    BTE_Alpha_Blending                       0x08006e6f   Thumb Code   124  lt738_lib.o(.text)
    LT738_PWM0_Init                          0x08006eeb   Thumb Code    86  lt738_lib.o(.text)
    LT738_PWM0_Duty                          0x08006f41   Thumb Code    12  lt738_lib.o(.text)
    LT738_PWM1_Init                          0x08006f4d   Thumb Code    86  lt738_lib.o(.text)
    LT738_PWM1_Duty                          0x08006fa3   Thumb Code    12  lt738_lib.o(.text)
    LT738_Standby                            0x08006faf   Thumb Code    12  lt738_lib.o(.text)
    LT738_Wkup_Standby                       0x08006fbb   Thumb Code    12  lt738_lib.o(.text)
    LT738_Suspend                            0x08006fc7   Thumb Code    18  lt738_lib.o(.text)
    LT738_Wkup_Suspend                       0x08006fd9   Thumb Code    20  lt738_lib.o(.text)
    LT738_SleepMode                          0x08006fed   Thumb Code    12  lt738_lib.o(.text)
    LT738_Wkup_Sleep                         0x08006ff9   Thumb Code    12  lt738_lib.o(.text)
    MPU_Memory_Write_Window_8bit             0x08007005   Thumb Code   148  lt738_lib.o(.text)
    MPU_Memory_Write_Pixel_8bit              0x08007099   Thumb Code    94  lt738_lib.o(.text)
    GT9147_WR_Reg                            0x080070fd   Thumb Code    92  gt9147.o(.text)
    GT9147_Send_Cfg                          0x08007159   Thumb Code    80  gt9147.o(.text)
    GT9147_RD_Reg                            0x080071a9   Thumb Code    98  gt9147.o(.text)
    GT9147_Init                              0x0800720b   Thumb Code   246  gt9147.o(.text)
    GT9147_Scan                              0x08007301   Thumb Code   516  gt9147.o(.text)
    delay_init                               0x08007571   Thumb Code    52  delay.o(.text)
    delay_us                                 0x080075a5   Thumb Code    72  delay.o(.text)
    delay_xms                                0x080075ed   Thumb Code    72  delay.o(.text)
    delay_ms                                 0x08007635   Thumb Code    56  delay.o(.text)
    _sys_exit                                0x08007675   Thumb Code     4  usart.o(.text)
    fputc                                    0x08007679   Thumb Code    22  usart.o(.text)
    uart_init                                0x0800768f   Thumb Code   164  usart.o(.text)
    USART1_IRQHandler                        0x08007733   Thumb Code   122  usart.o(.text)
    Reset_Handler                            0x080077bd   Thumb Code     8  startup_stm32f40_41xxx.o(.text)
    ADC_IRQHandler                           0x080077d7   Thumb Code     0  startup_stm32f40_41xxx.o(.text)
    CAN1_RX0_IRQHandler                      0x080077d7   Thumb Code     0  startup_stm32f40_41xxx.o(.text)
    CAN1_RX1_IRQHandler                      0x080077d7   Thumb Code     0  startup_stm32f40_41xxx.o(.text)
    CAN1_SCE_IRQHandler                      0x080077d7   Thumb Code     0  startup_stm32f40_41xxx.o(.text)
    CAN1_TX_IRQHandler                       0x080077d7   Thumb Code     0  startup_stm32f40_41xxx.o(.text)
    CAN2_RX0_IRQHandler                      0x080077d7   Thumb Code     0  startup_stm32f40_41xxx.o(.text)
    CAN2_RX1_IRQHandler                      0x080077d7   Thumb Code     0  startup_stm32f40_41xxx.o(.text)
    CAN2_SCE_IRQHandler                      0x080077d7   Thumb Code     0  startup_stm32f40_41xxx.o(.text)
    CAN2_TX_IRQHandler                       0x080077d7   Thumb Code     0  startup_stm32f40_41xxx.o(.text)
    CRYP_IRQHandler                          0x080077d7   Thumb Code     0  startup_stm32f40_41xxx.o(.text)
    DCMI_IRQHandler                          0x080077d7   Thumb Code     0  startup_stm32f40_41xxx.o(.text)
    DMA1_Stream0_IRQHandler                  0x080077d7   Thumb Code     0  startup_stm32f40_41xxx.o(.text)
    DMA1_Stream1_IRQHandler                  0x080077d7   Thumb Code     0  startup_stm32f40_41xxx.o(.text)
    DMA1_Stream2_IRQHandler                  0x080077d7   Thumb Code     0  startup_stm32f40_41xxx.o(.text)
    DMA1_Stream3_IRQHandler                  0x080077d7   Thumb Code     0  startup_stm32f40_41xxx.o(.text)
    DMA1_Stream4_IRQHandler                  0x080077d7   Thumb Code     0  startup_stm32f40_41xxx.o(.text)
    DMA1_Stream5_IRQHandler                  0x080077d7   Thumb Code     0  startup_stm32f40_41xxx.o(.text)
    DMA1_Stream6_IRQHandler                  0x080077d7   Thumb Code     0  startup_stm32f40_41xxx.o(.text)
    DMA1_Stream7_IRQHandler                  0x080077d7   Thumb Code     0  startup_stm32f40_41xxx.o(.text)
    DMA2_Stream0_IRQHandler                  0x080077d7   Thumb Code     0  startup_stm32f40_41xxx.o(.text)
    DMA2_Stream1_IRQHandler                  0x080077d7   Thumb Code     0  startup_stm32f40_41xxx.o(.text)
    DMA2_Stream2_IRQHandler                  0x080077d7   Thumb Code     0  startup_stm32f40_41xxx.o(.text)
    DMA2_Stream3_IRQHandler                  0x080077d7   Thumb Code     0  startup_stm32f40_41xxx.o(.text)
    DMA2_Stream4_IRQHandler                  0x080077d7   Thumb Code     0  startup_stm32f40_41xxx.o(.text)
    DMA2_Stream5_IRQHandler                  0x080077d7   Thumb Code     0  startup_stm32f40_41xxx.o(.text)
    DMA2_Stream6_IRQHandler                  0x080077d7   Thumb Code     0  startup_stm32f40_41xxx.o(.text)
    DMA2_Stream7_IRQHandler                  0x080077d7   Thumb Code     0  startup_stm32f40_41xxx.o(.text)
    ETH_IRQHandler                           0x080077d7   Thumb Code     0  startup_stm32f40_41xxx.o(.text)
    ETH_WKUP_IRQHandler                      0x080077d7   Thumb Code     0  startup_stm32f40_41xxx.o(.text)
    EXTI0_IRQHandler                         0x080077d7   Thumb Code     0  startup_stm32f40_41xxx.o(.text)
    EXTI15_10_IRQHandler                     0x080077d7   Thumb Code     0  startup_stm32f40_41xxx.o(.text)
    EXTI1_IRQHandler                         0x080077d7   Thumb Code     0  startup_stm32f40_41xxx.o(.text)
    EXTI2_IRQHandler                         0x080077d7   Thumb Code     0  startup_stm32f40_41xxx.o(.text)
    EXTI3_IRQHandler                         0x080077d7   Thumb Code     0  startup_stm32f40_41xxx.o(.text)
    EXTI4_IRQHandler                         0x080077d7   Thumb Code     0  startup_stm32f40_41xxx.o(.text)
    EXTI9_5_IRQHandler                       0x080077d7   Thumb Code     0  startup_stm32f40_41xxx.o(.text)
    FLASH_IRQHandler                         0x080077d7   Thumb Code     0  startup_stm32f40_41xxx.o(.text)
    FPU_IRQHandler                           0x080077d7   Thumb Code     0  startup_stm32f40_41xxx.o(.text)
    FSMC_IRQHandler                          0x080077d7   Thumb Code     0  startup_stm32f40_41xxx.o(.text)
    HASH_RNG_IRQHandler                      0x080077d7   Thumb Code     0  startup_stm32f40_41xxx.o(.text)
    I2C1_ER_IRQHandler                       0x080077d7   Thumb Code     0  startup_stm32f40_41xxx.o(.text)
    I2C1_EV_IRQHandler                       0x080077d7   Thumb Code     0  startup_stm32f40_41xxx.o(.text)
    I2C2_ER_IRQHandler                       0x080077d7   Thumb Code     0  startup_stm32f40_41xxx.o(.text)
    I2C2_EV_IRQHandler                       0x080077d7   Thumb Code     0  startup_stm32f40_41xxx.o(.text)
    I2C3_ER_IRQHandler                       0x080077d7   Thumb Code     0  startup_stm32f40_41xxx.o(.text)
    I2C3_EV_IRQHandler                       0x080077d7   Thumb Code     0  startup_stm32f40_41xxx.o(.text)
    OTG_FS_IRQHandler                        0x080077d7   Thumb Code     0  startup_stm32f40_41xxx.o(.text)
    OTG_FS_WKUP_IRQHandler                   0x080077d7   Thumb Code     0  startup_stm32f40_41xxx.o(.text)
    OTG_HS_EP1_IN_IRQHandler                 0x080077d7   Thumb Code     0  startup_stm32f40_41xxx.o(.text)
    OTG_HS_EP1_OUT_IRQHandler                0x080077d7   Thumb Code     0  startup_stm32f40_41xxx.o(.text)
    OTG_HS_IRQHandler                        0x080077d7   Thumb Code     0  startup_stm32f40_41xxx.o(.text)
    OTG_HS_WKUP_IRQHandler                   0x080077d7   Thumb Code     0  startup_stm32f40_41xxx.o(.text)
    PVD_IRQHandler                           0x080077d7   Thumb Code     0  startup_stm32f40_41xxx.o(.text)
    RCC_IRQHandler                           0x080077d7   Thumb Code     0  startup_stm32f40_41xxx.o(.text)
    RTC_Alarm_IRQHandler                     0x080077d7   Thumb Code     0  startup_stm32f40_41xxx.o(.text)
    RTC_WKUP_IRQHandler                      0x080077d7   Thumb Code     0  startup_stm32f40_41xxx.o(.text)
    SDIO_IRQHandler                          0x080077d7   Thumb Code     0  startup_stm32f40_41xxx.o(.text)
    SPI1_IRQHandler                          0x080077d7   Thumb Code     0  startup_stm32f40_41xxx.o(.text)
    SPI2_IRQHandler                          0x080077d7   Thumb Code     0  startup_stm32f40_41xxx.o(.text)
    SPI3_IRQHandler                          0x080077d7   Thumb Code     0  startup_stm32f40_41xxx.o(.text)
    TAMP_STAMP_IRQHandler                    0x080077d7   Thumb Code     0  startup_stm32f40_41xxx.o(.text)
    TIM1_BRK_TIM9_IRQHandler                 0x080077d7   Thumb Code     0  startup_stm32f40_41xxx.o(.text)
    TIM1_CC_IRQHandler                       0x080077d7   Thumb Code     0  startup_stm32f40_41xxx.o(.text)
    TIM1_TRG_COM_TIM11_IRQHandler            0x080077d7   Thumb Code     0  startup_stm32f40_41xxx.o(.text)
    TIM1_UP_TIM10_IRQHandler                 0x080077d7   Thumb Code     0  startup_stm32f40_41xxx.o(.text)
    TIM2_IRQHandler                          0x080077d7   Thumb Code     0  startup_stm32f40_41xxx.o(.text)
    TIM3_IRQHandler                          0x080077d7   Thumb Code     0  startup_stm32f40_41xxx.o(.text)
    TIM4_IRQHandler                          0x080077d7   Thumb Code     0  startup_stm32f40_41xxx.o(.text)
    TIM5_IRQHandler                          0x080077d7   Thumb Code     0  startup_stm32f40_41xxx.o(.text)
    TIM6_DAC_IRQHandler                      0x080077d7   Thumb Code     0  startup_stm32f40_41xxx.o(.text)
    TIM7_IRQHandler                          0x080077d7   Thumb Code     0  startup_stm32f40_41xxx.o(.text)
    TIM8_BRK_TIM12_IRQHandler                0x080077d7   Thumb Code     0  startup_stm32f40_41xxx.o(.text)
    TIM8_CC_IRQHandler                       0x080077d7   Thumb Code     0  startup_stm32f40_41xxx.o(.text)
    TIM8_TRG_COM_TIM14_IRQHandler            0x080077d7   Thumb Code     0  startup_stm32f40_41xxx.o(.text)
    TIM8_UP_TIM13_IRQHandler                 0x080077d7   Thumb Code     0  startup_stm32f40_41xxx.o(.text)
    UART4_IRQHandler                         0x080077d7   Thumb Code     0  startup_stm32f40_41xxx.o(.text)
    UART5_IRQHandler                         0x080077d7   Thumb Code     0  startup_stm32f40_41xxx.o(.text)
    USART2_IRQHandler                        0x080077d7   Thumb Code     0  startup_stm32f40_41xxx.o(.text)
    USART3_IRQHandler                        0x080077d7   Thumb Code     0  startup_stm32f40_41xxx.o(.text)
    USART6_IRQHandler                        0x080077d7   Thumb Code     0  startup_stm32f40_41xxx.o(.text)
    WWDG_IRQHandler                          0x080077d7   Thumb Code     0  startup_stm32f40_41xxx.o(.text)
    __user_initial_stackheap                 0x080077d9   Thumb Code     0  startup_stm32f40_41xxx.o(.text)
    NVIC_PriorityGroupConfig                 0x080077fd   Thumb Code    10  misc.o(.text)
    NVIC_Init                                0x08007807   Thumb Code   106  misc.o(.text)
    NVIC_SetVectorTable                      0x08007871   Thumb Code    14  misc.o(.text)
    NVIC_SystemLPConfig                      0x0800787f   Thumb Code    34  misc.o(.text)
    SysTick_CLKSourceConfig                  0x080078a1   Thumb Code    40  misc.o(.text)
    GPIO_DeInit                              0x080078dd   Thumb Code   268  stm32f4xx_gpio.o(.text)
    GPIO_Init                                0x080079e9   Thumb Code   144  stm32f4xx_gpio.o(.text)
    GPIO_StructInit                          0x08007a79   Thumb Code    18  stm32f4xx_gpio.o(.text)
    GPIO_PinLockConfig                       0x08007a8b   Thumb Code    34  stm32f4xx_gpio.o(.text)
    GPIO_ReadInputDataBit                    0x08007aad   Thumb Code    18  stm32f4xx_gpio.o(.text)
    GPIO_ReadInputData                       0x08007abf   Thumb Code     8  stm32f4xx_gpio.o(.text)
    GPIO_ReadOutputDataBit                   0x08007ac7   Thumb Code    18  stm32f4xx_gpio.o(.text)
    GPIO_ReadOutputData                      0x08007ad9   Thumb Code     8  stm32f4xx_gpio.o(.text)
    GPIO_SetBits                             0x08007ae1   Thumb Code     4  stm32f4xx_gpio.o(.text)
    GPIO_ResetBits                           0x08007ae5   Thumb Code     4  stm32f4xx_gpio.o(.text)
    GPIO_WriteBit                            0x08007ae9   Thumb Code    10  stm32f4xx_gpio.o(.text)
    GPIO_Write                               0x08007af3   Thumb Code     4  stm32f4xx_gpio.o(.text)
    GPIO_ToggleBits                          0x08007af7   Thumb Code     8  stm32f4xx_gpio.o(.text)
    GPIO_PinAFConfig                         0x08007aff   Thumb Code    70  stm32f4xx_gpio.o(.text)
    FSMC_NORSRAMDeInit                       0x08007b71   Thumb Code    54  stm32f4xx_fsmc.o(.text)
    FSMC_NORSRAMInit                         0x08007ba7   Thumb Code   230  stm32f4xx_fsmc.o(.text)
    FSMC_NORSRAMStructInit                   0x08007c8d   Thumb Code    48  stm32f4xx_fsmc.o(.text)
    FSMC_NORSRAMCmd                          0x08007cbd   Thumb Code    46  stm32f4xx_fsmc.o(.text)
    FSMC_NANDDeInit                          0x08007ceb   Thumb Code    62  stm32f4xx_fsmc.o(.text)
    FSMC_NANDInit                            0x08007d29   Thumb Code   132  stm32f4xx_fsmc.o(.text)
    FSMC_NANDStructInit                      0x08007dad   Thumb Code    54  stm32f4xx_fsmc.o(.text)
    FSMC_NANDCmd                             0x08007de3   Thumb Code    86  stm32f4xx_fsmc.o(.text)
    FSMC_NANDECCCmd                          0x08007e39   Thumb Code    86  stm32f4xx_fsmc.o(.text)
    FSMC_GetECC                              0x08007e8f   Thumb Code    24  stm32f4xx_fsmc.o(.text)
    FSMC_PCCARDDeInit                        0x08007ea7   Thumb Code    36  stm32f4xx_fsmc.o(.text)
    FSMC_PCCARDInit                          0x08007ecb   Thumb Code   130  stm32f4xx_fsmc.o(.text)
    FSMC_PCCARDStructInit                    0x08007f4d   Thumb Code    60  stm32f4xx_fsmc.o(.text)
    FSMC_PCCARDCmd                           0x08007f89   Thumb Code    44  stm32f4xx_fsmc.o(.text)
    FSMC_ITConfig                            0x08007fb5   Thumb Code   128  stm32f4xx_fsmc.o(.text)
    FSMC_GetFlagStatus                       0x08008035   Thumb Code    54  stm32f4xx_fsmc.o(.text)
    FSMC_ClearFlag                           0x0800806b   Thumb Code    74  stm32f4xx_fsmc.o(.text)
    FSMC_GetITStatus                         0x080080b5   Thumb Code    62  stm32f4xx_fsmc.o(.text)
    FSMC_ClearITPendingBit                   0x080080f3   Thumb Code    66  stm32f4xx_fsmc.o(.text)
    RCC_DeInit                               0x08008139   Thumb Code    82  stm32f4xx_rcc.o(.text)
    RCC_HSEConfig                            0x0800818b   Thumb Code    14  stm32f4xx_rcc.o(.text)
    RCC_GetFlagStatus                        0x08008199   Thumb Code    60  stm32f4xx_rcc.o(.text)
    RCC_WaitForHSEStartUp                    0x080081d5   Thumb Code    56  stm32f4xx_rcc.o(.text)
    RCC_AdjustHSICalibrationValue            0x0800820d   Thumb Code    20  stm32f4xx_rcc.o(.text)
    RCC_HSICmd                               0x08008221   Thumb Code     6  stm32f4xx_rcc.o(.text)
    RCC_LSEConfig                            0x08008227   Thumb Code    46  stm32f4xx_rcc.o(.text)
    RCC_LSICmd                               0x08008255   Thumb Code     6  stm32f4xx_rcc.o(.text)
    RCC_PLLConfig                            0x0800825b   Thumb Code    32  stm32f4xx_rcc.o(.text)
    RCC_PLLCmd                               0x0800827b   Thumb Code     6  stm32f4xx_rcc.o(.text)
    RCC_PLLI2SConfig                         0x08008281   Thumb Code    14  stm32f4xx_rcc.o(.text)
    RCC_PLLI2SCmd                            0x0800828f   Thumb Code     6  stm32f4xx_rcc.o(.text)
    RCC_PLLSAIConfig                         0x08008295   Thumb Code    20  stm32f4xx_rcc.o(.text)
    RCC_PLLSAICmd                            0x080082a9   Thumb Code     6  stm32f4xx_rcc.o(.text)
    RCC_ClockSecuritySystemCmd               0x080082af   Thumb Code     6  stm32f4xx_rcc.o(.text)
    RCC_MCO1Config                           0x080082b5   Thumb Code    28  stm32f4xx_rcc.o(.text)
    RCC_MCO2Config                           0x080082d1   Thumb Code    28  stm32f4xx_rcc.o(.text)
    RCC_SYSCLKConfig                         0x080082ed   Thumb Code    20  stm32f4xx_rcc.o(.text)
    RCC_GetSYSCLKSource                      0x08008301   Thumb Code    12  stm32f4xx_rcc.o(.text)
    RCC_HCLKConfig                           0x0800830d   Thumb Code    20  stm32f4xx_rcc.o(.text)
    RCC_PCLK1Config                          0x08008321   Thumb Code    20  stm32f4xx_rcc.o(.text)
    RCC_PCLK2Config                          0x08008335   Thumb Code    22  stm32f4xx_rcc.o(.text)
    RCC_GetClocksFreq                        0x0800834b   Thumb Code   222  stm32f4xx_rcc.o(.text)
    RCC_RTCCLKConfig                         0x08008429   Thumb Code    54  stm32f4xx_rcc.o(.text)
    RCC_RTCCLKCmd                            0x0800845f   Thumb Code     8  stm32f4xx_rcc.o(.text)
    RCC_BackupResetCmd                       0x08008467   Thumb Code     8  stm32f4xx_rcc.o(.text)
    RCC_I2SCLKConfig                         0x0800846f   Thumb Code     6  stm32f4xx_rcc.o(.text)
    RCC_SAIPLLI2SClkDivConfig                0x08008475   Thumb Code    26  stm32f4xx_rcc.o(.text)
    RCC_SAIPLLSAIClkDivConfig                0x0800848f   Thumb Code    28  stm32f4xx_rcc.o(.text)
    RCC_SAIBlockACLKConfig                   0x080084ab   Thumb Code    20  stm32f4xx_rcc.o(.text)
    RCC_SAIBlockBCLKConfig                   0x080084bf   Thumb Code    20  stm32f4xx_rcc.o(.text)
    RCC_LTDCCLKDivConfig                     0x080084d3   Thumb Code    20  stm32f4xx_rcc.o(.text)
    RCC_TIMCLKPresConfig                     0x080084e7   Thumb Code     6  stm32f4xx_rcc.o(.text)
    RCC_AHB1PeriphClockCmd                   0x080084ed   Thumb Code    34  stm32f4xx_rcc.o(.text)
    RCC_AHB2PeriphClockCmd                   0x0800850f   Thumb Code    78  stm32f4xx_rcc.o(.text)
    RCC_AHB3PeriphClockCmd                   0x0800855d   Thumb Code    34  stm32f4xx_rcc.o(.text)
    RCC_APB1PeriphClockCmd                   0x0800857f   Thumb Code    34  stm32f4xx_rcc.o(.text)
    RCC_APB2PeriphClockCmd                   0x080085a1   Thumb Code    34  stm32f4xx_rcc.o(.text)
    RCC_AHB1PeriphResetCmd                   0x080085c3   Thumb Code    34  stm32f4xx_rcc.o(.text)
    RCC_AHB2PeriphResetCmd                   0x080085e5   Thumb Code    34  stm32f4xx_rcc.o(.text)
    RCC_AHB3PeriphResetCmd                   0x08008607   Thumb Code    34  stm32f4xx_rcc.o(.text)
    RCC_APB1PeriphResetCmd                   0x08008629   Thumb Code    34  stm32f4xx_rcc.o(.text)
    RCC_APB2PeriphResetCmd                   0x0800864b   Thumb Code    34  stm32f4xx_rcc.o(.text)
    RCC_AHB1PeriphClockLPModeCmd             0x0800866d   Thumb Code    34  stm32f4xx_rcc.o(.text)
    RCC_AHB2PeriphClockLPModeCmd             0x0800868f   Thumb Code    34  stm32f4xx_rcc.o(.text)
    RCC_AHB3PeriphClockLPModeCmd             0x080086b1   Thumb Code    34  stm32f4xx_rcc.o(.text)
    RCC_APB1PeriphClockLPModeCmd             0x080086d3   Thumb Code    34  stm32f4xx_rcc.o(.text)
    RCC_APB2PeriphClockLPModeCmd             0x080086f5   Thumb Code    34  stm32f4xx_rcc.o(.text)
    RCC_LSEModeConfig                        0x08008717   Thumb Code    40  stm32f4xx_rcc.o(.text)
    RCC_ITConfig                             0x0800873f   Thumb Code    34  stm32f4xx_rcc.o(.text)
    RCC_ClearFlag                            0x08008761   Thumb Code    18  stm32f4xx_rcc.o(.text)
    RCC_GetITStatus                          0x08008773   Thumb Code    22  stm32f4xx_rcc.o(.text)
    RCC_ClearITPendingBit                    0x08008789   Thumb Code     8  stm32f4xx_rcc.o(.text)
    USART_DeInit                             0x08008795   Thumb Code   206  stm32f4xx_usart.o(.text)
    USART_Init                               0x08008863   Thumb Code   204  stm32f4xx_usart.o(.text)
    USART_StructInit                         0x0800892f   Thumb Code    24  stm32f4xx_usart.o(.text)
    USART_ClockInit                          0x08008947   Thumb Code    32  stm32f4xx_usart.o(.text)
    USART_ClockStructInit                    0x08008967   Thumb Code    12  stm32f4xx_usart.o(.text)
    USART_Cmd                                0x08008973   Thumb Code    24  stm32f4xx_usart.o(.text)
    USART_SetPrescaler                       0x0800898b   Thumb Code    16  stm32f4xx_usart.o(.text)
    USART_OverSampling8Cmd                   0x0800899b   Thumb Code    22  stm32f4xx_usart.o(.text)
    USART_OneBitMethodCmd                    0x080089b1   Thumb Code    24  stm32f4xx_usart.o(.text)
    USART_SendData                           0x080089c9   Thumb Code     8  stm32f4xx_usart.o(.text)
    USART_ReceiveData                        0x080089d1   Thumb Code    10  stm32f4xx_usart.o(.text)
    USART_SetAddress                         0x080089db   Thumb Code    18  stm32f4xx_usart.o(.text)
    USART_ReceiverWakeUpCmd                  0x080089ed   Thumb Code    24  stm32f4xx_usart.o(.text)
    USART_WakeUpConfig                       0x08008a05   Thumb Code    18  stm32f4xx_usart.o(.text)
    USART_LINBreakDetectLengthConfig         0x08008a17   Thumb Code    18  stm32f4xx_usart.o(.text)
    USART_LINCmd                             0x08008a29   Thumb Code    24  stm32f4xx_usart.o(.text)
    USART_SendBreak                          0x08008a41   Thumb Code    10  stm32f4xx_usart.o(.text)
    USART_HalfDuplexCmd                      0x08008a4b   Thumb Code    24  stm32f4xx_usart.o(.text)
    USART_SetGuardTime                       0x08008a63   Thumb Code    16  stm32f4xx_usart.o(.text)
    USART_SmartCardCmd                       0x08008a73   Thumb Code    24  stm32f4xx_usart.o(.text)
    USART_SmartCardNACKCmd                   0x08008a8b   Thumb Code    24  stm32f4xx_usart.o(.text)
    USART_IrDAConfig                         0x08008aa3   Thumb Code    18  stm32f4xx_usart.o(.text)
    USART_IrDACmd                            0x08008ab5   Thumb Code    24  stm32f4xx_usart.o(.text)
    USART_DMACmd                             0x08008acd   Thumb Code    18  stm32f4xx_usart.o(.text)
    USART_ITConfig                           0x08008adf   Thumb Code    74  stm32f4xx_usart.o(.text)
    USART_GetFlagStatus                      0x08008b29   Thumb Code    26  stm32f4xx_usart.o(.text)
    USART_ClearFlag                          0x08008b43   Thumb Code    18  stm32f4xx_usart.o(.text)
    USART_GetITStatus                        0x08008b55   Thumb Code   118  stm32f4xx_usart.o(.text)
    USART_ClearITPendingBit                  0x08008bcb   Thumb Code    30  stm32f4xx_usart.o(.text)
    __use_no_semihosting                     0x08008be9   Thumb Code     2  use_no_semi_2.o(.text)
    __2printf                                0x08008bed   Thumb Code    20  noretval__2printf.o(.text)
    _printf_str                              0x08008c05   Thumb Code    82  _printf_str.o(.text)
    _printf_int_dec                          0x08008c59   Thumb Code   104  _printf_dec.o(.text)
    _printf_int_hex                          0x08008cd1   Thumb Code    84  _printf_hex_int.o(.text)
    _printf_longlong_hex                     0x08008cd1   Thumb Code     0  _printf_hex_int.o(.text)
    __printf                                 0x08008d29   Thumb Code   308  __printf_flags_wp.o(.text)
    __aeabi_memclr4                          0x08008e61   Thumb Code     0  rt_memclr_w.o(.text)
    __aeabi_memclr8                          0x08008e61   Thumb Code     0  rt_memclr_w.o(.text)
    __rt_memclr_w                            0x08008e61   Thumb Code    78  rt_memclr_w.o(.text)
    _memset_w                                0x08008e65   Thumb Code     0  rt_memclr_w.o(.text)
    strcmp                                   0x08008eb1   Thumb Code   128  strcmpv7m.o(.text)
    __use_two_region_memory                  0x08008f31   Thumb Code     2  heapauxi.o(.text)
    __rt_heap_escrow$2region                 0x08008f33   Thumb Code     2  heapauxi.o(.text)
    __rt_heap_expand$2region                 0x08008f35   Thumb Code     2  heapauxi.o(.text)
    __I$use$semihosting                      0x08008f37   Thumb Code     0  use_no_semi.o(.text)
    __use_no_semihosting_swi                 0x08008f37   Thumb Code     2  use_no_semi.o(.text)
    __read_errno                             0x08008f39   Thumb Code    10  _rserrno.o(.text)
    __set_errno                              0x08008f43   Thumb Code    12  _rserrno.o(.text)
    _printf_int_common                       0x08008f4f   Thumb Code   178  _printf_intcommon.o(.text)
    _printf_cs_common                        0x08009001   Thumb Code    20  _printf_char.o(.text)
    _printf_char                             0x08009015   Thumb Code    16  _printf_char.o(.text)
    _printf_string                           0x08009025   Thumb Code     8  _printf_char.o(.text)
    _printf_char_file                        0x0800902d   Thumb Code    32  _printf_char_file.o(.text)
    __aeabi_errno_addr                       0x08009051   Thumb Code     8  rt_errno_addr_intlibspace.o(.text)
    __errno$intlibspace                      0x08009051   Thumb Code     0  rt_errno_addr_intlibspace.o(.text)
    __rt_errno_addr$intlibspace              0x08009051   Thumb Code     0  rt_errno_addr_intlibspace.o(.text)
    _printf_char_common                      0x08009063   Thumb Code    32  _printf_char_common.o(.text)
    ferror                                   0x08009089   Thumb Code     8  ferror.o(.text)
    __user_libspace                          0x08009091   Thumb Code     8  libspace.o(.text)
    __user_perproc_libspace                  0x08009091   Thumb Code     0  libspace.o(.text)
    __user_perthread_libspace                0x08009091   Thumb Code     0  libspace.o(.text)
    __user_setup_stackheap                   0x08009099   Thumb Code    74  sys_stackheap_outer.o(.text)
    exit                                     0x080090e3   Thumb Code    18  exit.o(.text)
    __hardfp_sqrt                            0x080090f5   Thumb Code   122  sqrt.o(i.__hardfp_sqrt)
    _is_digit                                0x0800916f   Thumb Code    14  __printf_wp.o(i._is_digit)
    __aeabi_dneg                             0x0800917d   Thumb Code     0  basic.o(x$fpl$basic)
    _dneg                                    0x0800917d   Thumb Code     6  basic.o(x$fpl$basic)
    __aeabi_fneg                             0x08009183   Thumb Code     0  basic.o(x$fpl$basic)
    _fneg                                    0x08009183   Thumb Code     6  basic.o(x$fpl$basic)
    _dabs                                    0x08009189   Thumb Code     6  basic.o(x$fpl$basic)
    _fabs                                    0x0800918f   Thumb Code     6  basic.o(x$fpl$basic)
    __fpl_dcmp_Inf                           0x08009195   Thumb Code    24  dcmpi.o(x$fpl$dcmpinf)
    __aeabi_ddiv                             0x080091ad   Thumb Code     0  ddiv.o(x$fpl$ddiv)
    _ddiv                                    0x080091ad   Thumb Code   552  ddiv.o(x$fpl$ddiv)
    __aeabi_d2uiz                            0x0800945d   Thumb Code     0  dfixu.o(x$fpl$dfixu)
    _dfixu                                   0x0800945d   Thumb Code    90  dfixu.o(x$fpl$dfixu)
    __aeabi_i2d                              0x080094b7   Thumb Code     0  dflt_clz.o(x$fpl$dflt)
    _dflt                                    0x080094b7   Thumb Code    46  dflt_clz.o(x$fpl$dflt)
    __aeabi_ui2d                             0x080094e5   Thumb Code     0  dflt_clz.o(x$fpl$dfltu)
    _dfltu                                   0x080094e5   Thumb Code    38  dflt_clz.o(x$fpl$dfltu)
    __aeabi_cdcmple                          0x0800950d   Thumb Code     0  dleqf.o(x$fpl$dleqf)
    _dcmple                                  0x0800950d   Thumb Code   120  dleqf.o(x$fpl$dleqf)
    __fpl_dcmple_InfNaN                      0x0800956f   Thumb Code     0  dleqf.o(x$fpl$dleqf)
    __aeabi_dmul                             0x08009585   Thumb Code     0  dmul.o(x$fpl$dmul)
    _dmul                                    0x08009585   Thumb Code   332  dmul.o(x$fpl$dmul)
    __fpl_dnaninf                            0x080096d9   Thumb Code   156  dnaninf.o(x$fpl$dnaninf)
    __fpl_dretinf                            0x08009775   Thumb Code    12  dretinf.o(x$fpl$dretinf)
    __aeabi_cdrcmple                         0x08009781   Thumb Code     0  drleqf.o(x$fpl$drleqf)
    _drcmple                                 0x08009781   Thumb Code   108  drleqf.o(x$fpl$drleqf)
    _dsqrt                                   0x080097ed   Thumb Code   404  dsqrt_umaal.o(x$fpl$dsqrt)
    __aeabi_f2d                              0x08009985   Thumb Code     0  f2d.o(x$fpl$f2d)
    _f2d                                     0x08009985   Thumb Code    86  f2d.o(x$fpl$f2d)
    __fpl_fnaninf                            0x080099db   Thumb Code   140  fnaninf.o(x$fpl$fnaninf)
    _fp_init                                 0x08009a67   Thumb Code    10  fpinit.o(x$fpl$fpinit)
    __fplib_config_fpu_vfp                   0x08009a6f   Thumb Code     0  fpinit.o(x$fpl$fpinit)
    __fplib_config_pureend_doubles           0x08009a6f   Thumb Code     0  fpinit.o(x$fpl$fpinit)
    POINT_COLOR_TBL                          0x08009a70   Data          10  main.o(.constdata)
    __I$use$fp                               0x08009a70   Number         0  usenofp.o(x$fpl$usenofp)
    pic                                      0x08009a7a   Data         464  main.o(.constdata)
    pic1                                     0x08009c4a   Data           2  main.o(.constdata)
    pic2                                     0x08009c4c   Data           2  main.o(.constdata)
    asc2_1206                                0x08009c4e   Data        1140  touch.o(.constdata)
    asc2_1608                                0x0800a0c2   Data        1520  touch.o(.constdata)
    asc2_2412                                0x0800a6b2   Data        3420  touch.o(.constdata)
    gImage_home480272                        0x0800b40e   Data       261120  gimage_home480272.o(.constdata)
    GT9147_CFG_TBL                           0x0804b00e   Data         186  gt9147.o(.constdata)
    GT9147_TPX_TBL                           0x0804b0c8   Data          10  gt9147.o(.constdata)
    FSMC_DefaultTimingStruct                 0x0804b0d4   Data          28  stm32f4xx_fsmc.o(.constdata)
    Region$$Table$$Base                      0x0804b1a8   Number         0  anon$$obj.o(Region$$Table)
    Region$$Table$$Limit                     0x0804b1c8   Number         0  anon$$obj.o(Region$$Table)
    SystemCoreClock                          0x20000000   Data           4  system_stm32f4xx.o(.data)
    AHBPrescTable                            0x20000004   Data          16  system_stm32f4xx.o(.data)
    tp_dev                                   0x20000018   Data          52  touch.o(.data)
    CMD_RDX                                  0x2000004c   Data           1  touch.o(.data)
    CMD_RDY                                  0x2000004d   Data           1  touch.o(.data)
    CCLK                                     0x2000004e   Data           1  lt738_lib.o(.data)
    MCLK                                     0x2000004f   Data           1  lt738_lib.o(.data)
    SCLK                                     0x20000050   Data           1  lt738_lib.o(.data)
    __stdout                                 0x20000058   Data           4  usart.o(.data)
    USART_RX_STA                             0x2000005c   Data           2  usart.o(.data)
    USART_RX_BUF                             0x20000070   Data         200  usart.o(.bss)
    __libspace_start                         0x20000138   Data          96  libspace.o(.bss)
    __temporary_stack_top$libspace           0x20000198   Data           0  libspace.o(.bss)



==============================================================================

Memory Map of the image

  Image Entry point : 0x08000189

  Load Region LR_IROM1 (Base: 0x08000000, Size: 0x0004b238, Max: 0x00100000, ABSOLUTE)

    Execution Region ER_IROM1 (Base: 0x08000000, Size: 0x0004b1c8, Max: 0x00100000, ABSOLUTE)

    Base Addr    Size         Type   Attr      Idx    E Section Name        Object

    0x08000000   0x00000188   Data   RO          639    RESET               startup_stm32f40_41xxx.o
    0x08000188   0x00000008   Code   RO          836  * !!!main             c_w.l(__main.o)
    0x08000190   0x00000034   Code   RO         1060    !!!scatter          c_w.l(__scatter.o)
    0x080001c4   0x0000001a   Code   RO         1062    !!handler_copy      c_w.l(__scatter_copy.o)
    0x080001de   0x00000002   PAD
    0x080001e0   0x0000001c   Code   RO         1064    !!handler_zi        c_w.l(__scatter_zi.o)
    0x080001fc   0x00000000   Code   RO          829    .ARM.Collect$$_printf_percent$$00000000  c_w.l(_printf_percent.o)
    0x080001fc   0x00000006   Code   RO          828    .ARM.Collect$$_printf_percent$$00000009  c_w.l(_printf_d.o)
    0x08000202   0x00000006   Code   RO          827    .ARM.Collect$$_printf_percent$$0000000C  c_w.l(_printf_x.o)
    0x08000208   0x00000006   Code   RO          826    .ARM.Collect$$_printf_percent$$00000014  c_w.l(_printf_s.o)
    0x0800020e   0x00000004   Code   RO          885    .ARM.Collect$$_printf_percent$$00000017  c_w.l(_printf_percent_end.o)
    0x08000212   0x00000002   Code   RO          937    .ARM.Collect$$libinit$$00000000  c_w.l(libinit.o)
    0x08000214   0x00000004   Code   RO          940    .ARM.Collect$$libinit$$00000001  c_w.l(libinit2.o)
    0x08000218   0x00000000   Code   RO          943    .ARM.Collect$$libinit$$00000004  c_w.l(libinit2.o)
    0x08000218   0x00000000   Code   RO          946    .ARM.Collect$$libinit$$0000000A  c_w.l(libinit2.o)
    0x08000218   0x00000000   Code   RO          948    .ARM.Collect$$libinit$$0000000C  c_w.l(libinit2.o)
    0x08000218   0x00000000   Code   RO          950    .ARM.Collect$$libinit$$0000000E  c_w.l(libinit2.o)
    0x08000218   0x00000000   Code   RO          953    .ARM.Collect$$libinit$$00000011  c_w.l(libinit2.o)
    0x08000218   0x00000000   Code   RO          955    .ARM.Collect$$libinit$$00000013  c_w.l(libinit2.o)
    0x08000218   0x00000000   Code   RO          957    .ARM.Collect$$libinit$$00000015  c_w.l(libinit2.o)
    0x08000218   0x00000000   Code   RO          959    .ARM.Collect$$libinit$$00000017  c_w.l(libinit2.o)
    0x08000218   0x00000000   Code   RO          961    .ARM.Collect$$libinit$$00000019  c_w.l(libinit2.o)
    0x08000218   0x00000000   Code   RO          963    .ARM.Collect$$libinit$$0000001B  c_w.l(libinit2.o)
    0x08000218   0x00000000   Code   RO          965    .ARM.Collect$$libinit$$0000001D  c_w.l(libinit2.o)
    0x08000218   0x00000000   Code   RO          967    .ARM.Collect$$libinit$$0000001F  c_w.l(libinit2.o)
    0x08000218   0x00000000   Code   RO          969    .ARM.Collect$$libinit$$00000021  c_w.l(libinit2.o)
    0x08000218   0x00000000   Code   RO          971    .ARM.Collect$$libinit$$00000023  c_w.l(libinit2.o)
    0x08000218   0x00000000   Code   RO          973    .ARM.Collect$$libinit$$00000025  c_w.l(libinit2.o)
    0x08000218   0x00000000   Code   RO          977    .ARM.Collect$$libinit$$0000002C  c_w.l(libinit2.o)
    0x08000218   0x00000000   Code   RO          979    .ARM.Collect$$libinit$$0000002E  c_w.l(libinit2.o)
    0x08000218   0x00000000   Code   RO          981    .ARM.Collect$$libinit$$00000030  c_w.l(libinit2.o)
    0x08000218   0x00000000   Code   RO          983    .ARM.Collect$$libinit$$00000032  c_w.l(libinit2.o)
    0x08000218   0x00000002   Code   RO          984    .ARM.Collect$$libinit$$00000033  c_w.l(libinit2.o)
    0x0800021a   0x00000002   Code   RO         1002    .ARM.Collect$$libshutdown$$00000000  c_w.l(libshutdown.o)
    0x0800021c   0x00000000   Code   RO         1012    .ARM.Collect$$libshutdown$$00000002  c_w.l(libshutdown2.o)
    0x0800021c   0x00000000   Code   RO         1014    .ARM.Collect$$libshutdown$$00000004  c_w.l(libshutdown2.o)
    0x0800021c   0x00000000   Code   RO         1017    .ARM.Collect$$libshutdown$$00000007  c_w.l(libshutdown2.o)
    0x0800021c   0x00000000   Code   RO         1020    .ARM.Collect$$libshutdown$$0000000A  c_w.l(libshutdown2.o)
    0x0800021c   0x00000000   Code   RO         1022    .ARM.Collect$$libshutdown$$0000000C  c_w.l(libshutdown2.o)
    0x0800021c   0x00000000   Code   RO         1025    .ARM.Collect$$libshutdown$$0000000F  c_w.l(libshutdown2.o)
    0x0800021c   0x00000002   Code   RO         1026    .ARM.Collect$$libshutdown$$00000010  c_w.l(libshutdown2.o)
    0x0800021e   0x00000000   Code   RO          876    .ARM.Collect$$rtentry$$00000000  c_w.l(__rtentry.o)
    0x0800021e   0x00000000   Code   RO          898    .ARM.Collect$$rtentry$$00000002  c_w.l(__rtentry2.o)
    0x0800021e   0x00000006   Code   RO          910    .ARM.Collect$$rtentry$$00000004  c_w.l(__rtentry4.o)
    0x08000224   0x00000000   Code   RO          900    .ARM.Collect$$rtentry$$00000009  c_w.l(__rtentry2.o)
    0x08000224   0x00000004   Code   RO          901    .ARM.Collect$$rtentry$$0000000A  c_w.l(__rtentry2.o)
    0x08000228   0x00000000   Code   RO          903    .ARM.Collect$$rtentry$$0000000C  c_w.l(__rtentry2.o)
    0x08000228   0x00000008   Code   RO          904    .ARM.Collect$$rtentry$$0000000D  c_w.l(__rtentry2.o)
    0x08000230   0x00000002   Code   RO          938    .ARM.Collect$$rtexit$$00000000  c_w.l(rtexit.o)
    0x08000232   0x00000000   Code   RO          986    .ARM.Collect$$rtexit$$00000002  c_w.l(rtexit2.o)
    0x08000232   0x00000004   Code   RO          987    .ARM.Collect$$rtexit$$00000003  c_w.l(rtexit2.o)
    0x08000236   0x00000006   Code   RO          988    .ARM.Collect$$rtexit$$00000004  c_w.l(rtexit2.o)
    0x0800023c   0x000004c0   Code   RO            3    .text               main.o
    0x080006fc   0x0000001a   Code   RO          173    .text               stm32f4xx_it.o
    0x08000716   0x00000002   PAD
    0x08000718   0x00000210   Code   RO          222    .text               system_stm32f4xx.o
    0x08000928   0x00000040   Code   RO          248    .text               led.o
    0x08000968   0x0000028c   Code   RO          268    .text               key.o
    0x08000bf4   0x00000338   Code   RO          289    .text               if_port.o
    0x08000f2c   0x0000025c   Code   RO          309    .text               myiic.o
    0x08001188   0x0000017a   Code   RO          332    .text               24cxx.o
    0x08001302   0x00000002   PAD
    0x08001304   0x00000254   Code   RO          355    .text               ctiic.o
    0x08001558   0x00001040   Code   RO          408    .text               touch.o
    0x08002598   0x00002d34   Code   RO          473    .text               lt738.o
    0x080052cc   0x000002a2   Code   RO          493    .text               lt738_demo.o
    0x0800556e   0x00000002   PAD
    0x08005570   0x00001b8c   Code   RO          513    .text               lt738_lib.o
    0x080070fc   0x00000474   Code   RO          544    .text               gt9147.o
    0x08007570   0x00000104   Code   RO          568    .text               delay.o
    0x08007674   0x00000148   Code   RO          608    .text               usart.o
    0x080077bc   0x00000040   Code   RO          640    .text               startup_stm32f40_41xxx.o
    0x080077fc   0x000000e0   Code   RO          646    .text               misc.o
    0x080078dc   0x00000294   Code   RO          666    .text               stm32f4xx_gpio.o
    0x08007b70   0x000005c8   Code   RO          686    .text               stm32f4xx_fsmc.o
    0x08008138   0x0000065c   Code   RO          709    .text               stm32f4xx_rcc.o
    0x08008794   0x00000454   Code   RO          751    .text               stm32f4xx_usart.o
    0x08008be8   0x00000002   Code   RO          771    .text               c_w.l(use_no_semi_2.o)
    0x08008bea   0x00000002   PAD
    0x08008bec   0x00000018   Code   RO          775    .text               c_w.l(noretval__2printf.o)
    0x08008c04   0x00000052   Code   RO          781    .text               c_w.l(_printf_str.o)
    0x08008c56   0x00000002   PAD
    0x08008c58   0x00000078   Code   RO          783    .text               c_w.l(_printf_dec.o)
    0x08008cd0   0x00000058   Code   RO          788    .text               c_w.l(_printf_hex_int.o)
    0x08008d28   0x00000138   Code   RO          818    .text               c_w.l(__printf_flags_wp.o)
    0x08008e60   0x0000004e   Code   RO          830    .text               c_w.l(rt_memclr_w.o)
    0x08008eae   0x00000002   PAD
    0x08008eb0   0x00000080   Code   RO          832    .text               c_w.l(strcmpv7m.o)
    0x08008f30   0x00000006   Code   RO          834    .text               c_w.l(heapauxi.o)
    0x08008f36   0x00000002   Code   RO          874    .text               c_w.l(use_no_semi.o)
    0x08008f38   0x00000016   Code   RO          877    .text               c_w.l(_rserrno.o)
    0x08008f4e   0x000000b2   Code   RO          879    .text               c_w.l(_printf_intcommon.o)
    0x08009000   0x0000002c   Code   RO          881    .text               c_w.l(_printf_char.o)
    0x0800902c   0x00000024   Code   RO          883    .text               c_w.l(_printf_char_file.o)
    0x08009050   0x00000008   Code   RO          915    .text               c_w.l(rt_errno_addr_intlibspace.o)
    0x08009058   0x00000030   Code   RO          917    .text               c_w.l(_printf_char_common.o)
    0x08009088   0x00000008   Code   RO          919    .text               c_w.l(ferror.o)
    0x08009090   0x00000008   Code   RO          923    .text               c_w.l(libspace.o)
    0x08009098   0x0000004a   Code   RO          926    .text               c_w.l(sys_stackheap_outer.o)
    0x080090e2   0x00000012   Code   RO          930    .text               c_w.l(exit.o)
    0x080090f4   0x0000007a   Code   RO          862    i.__hardfp_sqrt     m_wm.l(sqrt.o)
    0x0800916e   0x0000000e   Code   RO          816    i._is_digit         c_w.l(__printf_wp.o)
    0x0800917c   0x00000018   Code   RO          838    x$fpl$basic         fz_wm.l(basic.o)
    0x08009194   0x00000018   Code   RO          886    x$fpl$dcmpinf       fz_wm.l(dcmpi.o)
    0x080091ac   0x000002b0   Code   RO          841    x$fpl$ddiv          fz_wm.l(ddiv.o)
    0x0800945c   0x0000005a   Code   RO          844    x$fpl$dfixu         fz_wm.l(dfixu.o)
    0x080094b6   0x0000002e   Code   RO          849    x$fpl$dflt          fz_wm.l(dflt_clz.o)
    0x080094e4   0x00000026   Code   RO          848    x$fpl$dfltu         fz_wm.l(dflt_clz.o)
    0x0800950a   0x00000002   PAD
    0x0800950c   0x00000078   Code   RO          854    x$fpl$dleqf         fz_wm.l(dleqf.o)
    0x08009584   0x00000154   Code   RO          856    x$fpl$dmul          fz_wm.l(dmul.o)
    0x080096d8   0x0000009c   Code   RO          888    x$fpl$dnaninf       fz_wm.l(dnaninf.o)
    0x08009774   0x0000000c   Code   RO          890    x$fpl$dretinf       fz_wm.l(dretinf.o)
    0x08009780   0x0000006c   Code   RO          858    x$fpl$drleqf        fz_wm.l(drleqf.o)
    0x080097ec   0x00000198   Code   RO          892    x$fpl$dsqrt         fz_wm.l(dsqrt_umaal.o)
    0x08009984   0x00000056   Code   RO          860    x$fpl$f2d           fz_wm.l(f2d.o)
    0x080099da   0x0000008c   Code   RO          894    x$fpl$fnaninf       fz_wm.l(fnaninf.o)
    0x08009a66   0x0000000a   Code   RO          994    x$fpl$fpinit        fz_wm.l(fpinit.o)
    0x08009a70   0x00000000   Code   RO          896    x$fpl$usenofp       fz_wm.l(usenofp.o)
    0x08009a70   0x000001de   Data   RO            4    .constdata          main.o
    0x08009c4e   0x000017c0   Data   RO          409    .constdata          touch.o
    0x0800b40e   0x0003fc00   Data   RO          535    .constdata          gimage_home480272.o
    0x0804b00e   0x000000c4   Data   RO          545    .constdata          gt9147.o
    0x0804b0d2   0x00000002   PAD
    0x0804b0d4   0x0000001c   Data   RO          687    .constdata          stm32f4xx_fsmc.o
    0x0804b0f0   0x00000028   Data   RO          789    .constdata          c_w.l(_printf_hex_int.o)
    0x0804b118   0x00000011   Data   RO          819    .constdata          c_w.l(__printf_flags_wp.o)
    0x0804b129   0x00000003   PAD
    0x0804b12c   0x00000079   Data   RO          410    .conststring        touch.o
    0x0804b1a5   0x00000003   PAD
    0x0804b1a8   0x00000020   Data   RO         1058    Region$$Table       anon$$obj.o


    Execution Region RW_IRAM1 (Base: 0x20000000, Size: 0x00000798, Max: 0x00020000, ABSOLUTE)

    Base Addr    Size         Type   Attr      Idx    E Section Name        Object

    0x20000000   0x00000014   Data   RW          223    .data               system_stm32f4xx.o
    0x20000014   0x00000002   Data   RW          269    .data               key.o
    0x20000016   0x00000002   PAD
    0x20000018   0x00000036   Data   RW          411    .data               touch.o
    0x2000004e   0x00000003   Data   RW          515    .data               lt738_lib.o
    0x20000051   0x00000001   Data   RW          546    .data               gt9147.o
    0x20000052   0x00000004   Data   RW          569    .data               delay.o
    0x20000056   0x00000002   PAD
    0x20000058   0x00000006   Data   RW          610    .data               usart.o
    0x2000005e   0x00000010   Data   RW          710    .data               stm32f4xx_rcc.o
    0x2000006e   0x00000002   PAD
    0x20000070   0x000000c8   Zero   RW          609    .bss                usart.o
    0x20000138   0x00000060   Zero   RW          924    .bss                c_w.l(libspace.o)
    0x20000198   0x00000200   Zero   RW          638    HEAP                startup_stm32f40_41xxx.o
    0x20000398   0x00000400   Zero   RW          637    STACK               startup_stm32f40_41xxx.o


==============================================================================

Image component sizes


      Code (inc. data)   RO Data    RW Data    ZI Data      Debug   Object Name

       378          0          0          0          0       2882   24cxx.o
       596         24          0          0          0       2109   ctiic.o
       260          8          0          4          0       1549   delay.o
         0          0     261120          0          0        512   gimage_home480272.o
      1140        108        196          1          0       3246   gt9147.o
       824         52          0          0          0       3445   if_port.o
       652         18          0          2          0       2407   key.o
        64          4          0          0          0        555   led.o
     11572          0          0          0          0      70512   lt738.o
       674          0          0          0          0       1640   lt738_demo.o
      7052         70          0          3          0      37022   lt738_lib.o
      1216         48        478          0          0     273136   main.o
       224         20          0          0          0       1885   misc.o
       604         14          0          0          0       1948   myiic.o
        64         26        392          0       1536        864   startup_stm32f40_41xxx.o
      1480         18         28          0          0       5750   stm32f4xx_fsmc.o
       660         44          0          0          0       4225   stm32f4xx_gpio.o
        26          0          0          0          0       1254   stm32f4xx_it.o
      1628         52          0         16          0      13136   stm32f4xx_rcc.o
      1108         34          0          0          0       7948   stm32f4xx_usart.o
       528         46          0         20          0       1879   system_stm32f4xx.o
      4160        222       6201         54          0       8794   touch.o
       328         16          0          6        200       3390   usart.o

    ----------------------------------------------------------------------
     35244        824     268452        112       1736     450088   Object Totals
         0          0         32          0          0          0   (incl. Generated)
         6          0          5          6          0          0   (incl. Padding)

    ----------------------------------------------------------------------

      Code (inc. data)   RO Data    RW Data    ZI Data      Debug   Library Member Name

         8          0          0          0          0         68   __main.o
       312          4         17          0          0         92   __printf_flags_wp.o
        14          0          0          0          0         68   __printf_wp.o
         0          0          0          0          0          0   __rtentry.o
        12          0          0          0          0          0   __rtentry2.o
         6          0          0          0          0          0   __rtentry4.o
        52          8          0          0          0          0   __scatter.o
        26          0          0          0          0          0   __scatter_copy.o
        28          0          0          0          0          0   __scatter_zi.o
        44          0          0          0          0        108   _printf_char.o
        48          6          0          0          0         96   _printf_char_common.o
        36          4          0          0          0         80   _printf_char_file.o
         6          0          0          0          0          0   _printf_d.o
       120         16          0          0          0         92   _printf_dec.o
        88          4         40          0          0         88   _printf_hex_int.o
       178          0          0          0          0         88   _printf_intcommon.o
         0          0          0          0          0          0   _printf_percent.o
         4          0          0          0          0          0   _printf_percent_end.o
         6          0          0          0          0          0   _printf_s.o
        82          0          0          0          0         80   _printf_str.o
         6          0          0          0          0          0   _printf_x.o
        22          0          0          0          0        100   _rserrno.o
        18          0          0          0          0         80   exit.o
         8          0          0          0          0         68   ferror.o
         6          0          0          0          0        152   heapauxi.o
         2          0          0          0          0          0   libinit.o
         6          0          0          0          0          0   libinit2.o
         2          0          0          0          0          0   libshutdown.o
         2          0          0          0          0          0   libshutdown2.o
         8          4          0          0         96         68   libspace.o
        24          4          0          0          0         84   noretval__2printf.o
         8          4          0          0          0         68   rt_errno_addr_intlibspace.o
        78          0          0          0          0         80   rt_memclr_w.o
         2          0          0          0          0          0   rtexit.o
        10          0          0          0          0          0   rtexit2.o
       128          0          0          0          0         68   strcmpv7m.o
        74          0          0          0          0         80   sys_stackheap_outer.o
         2          0          0          0          0         68   use_no_semi.o
         2          0          0          0          0         68   use_no_semi_2.o
        24          0          0          0          0        164   basic.o
        24          0          0          0          0        116   dcmpi.o
       688        140          0          0          0        256   ddiv.o
        90          4          0          0          0        140   dfixu.o
        84          0          0          0          0        232   dflt_clz.o
       120          4          0          0          0        140   dleqf.o
       340         12          0          0          0        152   dmul.o
       156          4          0          0          0        140   dnaninf.o
        12          0          0          0          0        116   dretinf.o
       108          0          0          0          0        128   drleqf.o
       408         56          0          0          0        168   dsqrt_umaal.o
        86          4          0          0          0        132   f2d.o
       140          4          0          0          0        132   fnaninf.o
        10          0          0          0          0        116   fpinit.o
         0          0          0          0          0          0   usenofp.o
       122          0          0          0          0        148   sqrt.o

    ----------------------------------------------------------------------
      3900        282         60          0         96       4124   Library Totals
        10          0          3          0          0          0   (incl. Padding)

    ----------------------------------------------------------------------

      Code (inc. data)   RO Data    RW Data    ZI Data      Debug   Library Name

      1478         54         57          0         96       1844   c_w.l
      2290        228          0          0          0       2132   fz_wm.l
       122          0          0          0          0        148   m_wm.l

    ----------------------------------------------------------------------
      3900        282         60          0         96       4124   Library Totals

    ----------------------------------------------------------------------

==============================================================================


      Code (inc. data)   RO Data    RW Data    ZI Data      Debug   

     39144       1106     268512        112       1832     448276   Grand Totals
     39144       1106     268512        112       1832     448276   ELF Image Totals
     39144       1106     268512        112          0          0   ROM Totals

==============================================================================

    Total RO  Size (Code + RO Data)               307656 ( 300.45kB)
    Total RW  Size (RW Data + ZI Data)              1944 (   1.90kB)
    Total ROM Size (Code + RO Data + RW Data)     307768 ( 300.55kB)

==============================================================================

